:020000040800F2
:1000000038120020A101000811630008814800088F
:100010000D63000841110008AD7A000800000000DF
:10002000000000000000000000000000456700081C
:100030004D19000800000000C9630008216C000889
:10004000BB010008BB010008BB010008BB010008A0
:10005000BB010008BB010008BB010008BB01000890
:10006000BB010008BB010008BB010008BB01000880
:10007000BB01000851140008BB010008BB010008C7
:10008000BB010008BB010008BB010008BB01000860
:10009000BB010008BB010008BB010008BB01000850
:1000A000BB010008BB010008BB010008BB01000840
:1000B000ED6C0008FD6C0008BB010008BB010008E6
:1000C000BB010008BB010008BB010008BB01000820
:1000D000BB010008BB0100081D770008BB01000838
:1000E000BB010008BB010008BB010008BB01000800
:1000F000BB010008BB010008BB010008BB010008F0
:10010000BB010008BB010008BB010008BB010008DF
:1001100019720008BB0100080D6D00081D6D000874
:10012000BB010008BB010008BB010008BB010008BF
:10013000BB010008BB010008BB010008BB010008AF
:10014000BB010008BB010008BB010008BB0100089F
:10015000BB010008BB010008BB010008BB0100088F
:10016000BB010008BB010008BB010008BB0100087F
:10017000BB010008BB010008BB0100080000000033
:10018000BB010008BB010008DFF810D000F0B0FC94
:100190000048004735890008AFF30080381200207E
:1001A0000648804706480047FEE7FEE7FEE7FEE711
:1001B000FEE7FEE7FEE7FEE7FEE7FEE7D96C000894
:1001C000890100082DE9F05F0546002092469B4614
:1001D00088460646814640241BE02846414647465D
:1001E000224600F04AFB53465A46C01A914110D3AA
:1001F00011461846224600F031FB2D1A67EB010824
:100200004F4622460120002100F028FB17EB000991
:100210004E41201EA4F10104DFDC484631462A4647
:100220004346BDE8F09FD2B201E000F8012B491E21
:10023000FBD270470022F6E710B513460A46044683
:100240001946FFF7F0FF204610BD30B505462A4697
:100250000B4612F8010B13F8014B08B1A042F8D07D
:100260001CB1002802D06D1CF1E7284630BD10B546
:10027000044604E00B7800F8013B03B1491C521E10
:10028000F8D2204610BDCAB2401E10F8011F8A42A3
:1002900002D00029F9D100207047421C10F8011B40
:1002A0000029FBD1801A70470022CBB20178994215
:1002B00000D10246401C0029F8D1104670470000CA
:1002C0000FB400B58DB010A909900B9000914FF0BC
:1002D000FF300A9000200C900548069005480790D2
:1002E0006A4609A80F9900F0FFFA0DB05DF814FBFB
:1002F00005090008230900082DE9FF5F1D464FF09E
:10030000FF3BD5E9014691465F464FF00008A969D9
:100310007F1C01988847296A824688470028F6D1C1
:10032000BAF1FF3F0CD024F4C064002E19DD600642
:1003300014D5BAF12B0F09D0BAF12D0F0ED103E06D
:10034000584604B0BDE8F09F44F48064A9697F1C5E
:1003500001988847761E8246002E02DDBAF1300FE2
:1003600003D0B9F1000F26D032E0A969761E44F41B
:1003700000747F1C019888478246002E05DDBAF183
:10038000780F06D0BAF1580F03D0B9F1000F10D092
:100390001EE0B9F1000F02D0B9F1100F18D1A96910
:1003A000761E24F400747F1C019888478246102032
:1003B00002E0082000E00A20814609E008FB090865
:1003C000A969761E44F400747F1C01988847824610
:1003D000002E05DD4946504600F071FA0028EDDA9E
:1003E000E96901988847A00502D46FF00100A8E7E9
:1003F000E00725D1600613D5600502D5C8F10000DD
:1004000000E0404629680A1D2A600968220501D5D6
:10041000087015E0220701D5088011E008600FE0A0
:100420002868011D29600068210502D580F8008038
:1004300006E0210702D5A0F8008001E0C0F80080A6
:1004400038467EE72DE9FE4F804681EA0300C00F63
:100450000C46009021F0004123F00045B8EB02006B
:10046000A94105D24046214690461C460B4602460D
:1004700023F00040104347D0270DC7F30A00C3F311
:100480000A510290401A019040286BDAC3F313001E
:1004900040F4801B0098924620B10023D2EB030A5F
:1004A00063EB0B0B01985946C0F14002504600F037
:1004B000D5F906460D4650465946019A00F0EDF929
:1004C00010EB08006141002487EA115284EAE773C7
:1004D0001A4340D0009A62B3019A012A4FEA0752A8
:1004E00015DC001B61EB02014FF0004202EA0752EB
:1004F000CDE90042001C41F5801132462B4600F048
:1005000067FA03B0BDE8F08F40462146F9E7001BCB
:1005100061EB0201001C41F5801300185B412018BB
:10052000A2F5001747EB030140EAD570B6196D41FB
:1005300011E06D084FEA360645EAC0754FEA0752EA
:10054000001B61EB0201001C41F5801149084FEAD4
:1005500030000019514132462B4603B0BDE8F04F40
:1005600000F027BA0098012240000023D0EB0202DD
:1005700063EBE073009821464FEAE074B8EB0000AB
:1005800061EB0401E9E783F000435BE781F00041A0
:1005900058E72DE9FE4F81EA030404F0004421F0FE
:1005A000004100944FF0000B23F0004350EA010497
:1005B0005ED052EA03045BD0C3F30A54C1F30A5578
:1005C0002C44A4F2F3340194A0FB0254C1F31301B0
:1005D00041F48011C3F3130343F4801301FB02447D
:1005E00000FB034E840A970A44EA815447EA835782
:1005F000A4FB076802958D0A05FB07854FEA932C3B
:1006000004FB0C542705029D4FEA065847EA1637AB
:10061000B5EB08056EEB070C870E920E47EA8117C3
:1006200042EA8312A7FB0201B6EB0B0164EB000464
:100630002B0D43EA0C335E1844EB1C50DA4651464E
:10064000E7FB0201C5F313044FEA0B3343EA1453EB
:100650004FEA0432019C43EA0603A4F10C0402941D
:10066000009CCDE900B400F0B3F903B0BDE8F08F11
:1006700000200146F9E72DE9F04D81EA030404F07A
:10068000004B21F0004514464FF0000A23F00041D2
:1006900050EA050220D054EA01021DD0C5F30A57E2
:1006A0000246C5F31303C1F31300C1F30A5640F425
:1006B000801543F48013A7EB0608101BD64608F2FA
:1006C000FD3873EB050002D308F1010801E0921830
:1006D0005B41B8F1000F03DA00200146BDE8F08D60
:1006E00000204FF48011064684460EE0171B73EB82
:1006F000050705D3121B63EB050306434CEA010C07
:1007000049084FEA300092185B4150EA0107EDD1E9
:1007100052EA030012D082EA040083EA050108438A
:1007200005D0101BAB4106D20122002306E00022B7
:100730004FF0004302E06FF0010253101AEB060085
:100740004CEB085110EB0A0041EB0B01BDE8F04DFA
:1007500000F02FB90EB540F2334102910021CDE9EE
:1007600000110A460B4600F033F903B000BDC1F397
:100770000A5210B5C1F3130140F2FF3341F4801166
:100780009A4201DA002010BD40F233439A42A2F2AD
:10079000334203DC524200F070F810BD904010BDAF
:1007A00000F0004230F000400AD0C10D01F5607148
:1007B000C0F3160042EA0151C208400711437047D6
:1007C000002001467047000030B5041E71F100049E
:1007D00004DB4FF00044404264EB0101141E73F14E
:1007E000000405DB1C464FF00043524263EB040358
:1007F000994208BF904230BD01F0004330B421F06F
:10080000004150EA010206D00A0DA2F56072C1F360
:100810001301002A02DC30BC00207047440F44EA78
:10082000C104C100E01830BC00EBC25000F08AB82F
:1008300030B50B46014600202022012409E021FAB0
:1008400002F59D4205D303FA02F5491B04FA02F5AD
:100850002844151EA2F10102F1DC30BD202A04DB80
:10086000203A00FA02F1002070479140C2F12003C3
:1008700020FA03F3194390407047202A04DB203A02
:1008800021FA02F00021704721FA02F3D040C2F1B0
:1008900020029140084319467047202A06DBCB17F7
:1008A000203A41FA02F043EAE07306E041FA02F32B
:1008B000D040C2F1200291400843194670473A28BF
:1008C00000D2303820F02002412A01D3A2F13700B3
:1008D000884201D34FF0FF30704700000268114496
:1008E0001378016018467047D1600449516104498A
:1008F000116200211161114600F012B9DD080008F3
:10090000150B0008426842B1016811F8013B23B1A0
:10091000521EC0E90012184670470121C160881EAE
:10092000704742685AB1C368016843B983688B4213
:1009300005D0491E521CC0E90012002070474FF03C
:10094000FF3070470029A8BF7047401C490008BF0E
:1009500020F00100704710B4B0FA80FC00FA0CF0EF
:1009600050EA010404BF10BC704749B1CCF1200427
:1009700021FA04F411FA0CF118BF012121430843B4
:10098000A3EB0C01CB1D4FEA00614FEA102042BFE0
:10099000002010BC704700EBC35010440029A4BFD6
:1009A00010BC7047401C490008BF20F0010010BC7B
:1009B000704710B5141E73F1000408DA401C41F1B1
:1009C000000192185B411A4301D120F0010010BDD3
:1009D0002DE9F04D92469B4611B1B1FA81F202E049
:1009E000B0FA80F220329046FFF738FF04460F46F7
:1009F00040EA0A0041EA0B0153465A46084313D025
:100A0000114653EA010019D0C8F140025046FFF7E1
:100A100034FF05460E46504659464246FFF71EFF34
:100A2000084305D0012004E020463946BDE8F08D9A
:100A30000020054346EAE0762C4337430A986305D5
:100A4000E40AA0EB08000022FD0A44EA47540A30F9
:100A500002D500200146E9E7010510196941DDE9E9
:100A6000084500196941BDE8F04DA2E70EB5C10F78
:100A700080EAE0700844CA07002140F233438DE861
:100A80000E000A460B46FFF7A3FF03B000BDC1F3FB
:100A90000A52C1F3130140F2FF3341F480119A422C
:100AA00002DA00200146704740F233439A42A2F234
:100AB000334202DC5242FFF7E0BEFFF7CFBE000038
:100AC00030B5041E71F1000404DB4FF000444042D5
:100AD00064EB0101141E73F1000405DB1C464FF0AA
:100AE0000043524263EB04038B4208BF824230BD95
:100AF000064C074D06E0E06840F0010394E807006B
:100B000098471034AC42F6D3FFF742FBA88C00089C
:100B1000C88C0008C0B24FF4F05100F099B9000041
:100B20002DE9F34F8BB04FF0000801F10C000C469B
:100B30004FF0010B46460DF1080A01906269012150
:100B400001989047051E2DD0252D2CD0216A88476D
:100B5000C0B16269012101989047216A8847002845
:100B6000F7D1411E62690198904700E0761CA169A7
:100B70000B988847216A88470028F7D1E1690B98CC
:100B80008847DBE7A1690B9888470746A84201D14F
:100B9000761CD3E7E1690B9888477F1C02D1B8F136
:100BA000000F6FD047E1002762693D463946019842
:100BB00090472A2804D162690121019890470125B4
:100BC000DFF888926269012101989047A0F1300115
:100BD0000A290AD24F45E5DC07EB870100EB410704
:100BE000303FDFD445F01005ECE7E90601D46FF0A3
:100BF00000476C280AD04C2814D0682815D06A28E1
:100C00000DD074281CD07A281AD01DE06269012109
:100C1000019890476C2802D045F0040514E045F097
:100C200002050DE045F020050AE062690121019806
:100C30009047682802D045F0080505E045F40065B6
:100C40006269012101989047C4E9015765283DD0A8
:100C500019DC58287AD00CDC452837D004DC25284C
:100C600026D0412831D131E046282FD047282CD139
:100C70002CE05B2877D0612828D063287CD06428BA
:100C800023D15AE0D1E06F2848D008DC66281DD077
:100C900067281BD0692821D06E2816D127E070283C
:100CA00045D0732868D0752847D078280DD14DE0FD
:100CB000A1690B988847054625283FF469AFE1698B
:100CC0000B9888476D1C3FF46AAFB4E023466A4630
:100CD0006FF001000B99AFF300809FE045F04000FA
:100CE0006060A80723464FF0000236D43EE0E807D4
:100CF0007FF447AF2068011D21600068290501D5F8
:100D000006701BE7290701D5068017E7A90703D559
:100D1000F117C0E9006111E706600FE745F04000F8
:100D20006060A80723464FF0080216D41EE040F684
:100D30000E0125EA0100606016E045F040006060A9
:100D4000A80723464FF00A0207D40FE045F0400001
:100D50006060A80708D5234610226FF001000B99A8
:100D6000AFF300805AE007E0234610226FF0010045
:100D70000B99FFF7C1FA51E04FF000094F464B467F
:100D8000632802D05B2807D041E02079C00601D457
:100D90000120A06001273AE0626901210198904793
:100DA0005E2805D14FF001096269494601989047D4
:100DB000216939B900210A46534643F82120491CCC
:100DC0000829FADBB0B3216969B9C11700EBD16218
:100DD00053110AEB830122F01F02821A01200B68D3
:100DE000904003430B6062690121019890475D28A0
:100DF000E8D1B9F1000F09D00020514651F8202068
:100E0000D24341F82020401C0828F7DB02AB2246E1
:100E100000976FF001000B99AFF3008000280CDA07
:100E2000401C08D1BBF1000F05D04FF0FF300DB0D2
:100E3000BDE8F08FFFE74046F9E7E90701D108F187
:100E4000010806444FF0000B78E60000CCCCCC0C37
:100E50007F2801D9002208E0064A02EB5002C007B1
:100E6000127800D1120902F00F02012090400840D0
:100E700070470000308B000870B58C1810F8015BCB
:100E800015F0070301D110F8013B2A1106D110F823
:100E9000012B03E010F8016B01F8016B5B1EF9D127
:100EA0002B0705D40023521E0DD401F8013BFAE7AD
:100EB00010F8013BCB1A921C03E013F8015B01F818
:100EC000015B521EF9D5A142D8D3002070BD70B588
:100ED0000546AC6B206C00F0500050BB206C40F419
:100EE000007020642068806800F04050E8B9207EDF
:100EF000D8B92068C06A00F4700020B1206880680A
:100F000000F4806088B92068406820F020002168E3
:100F10004860206C20F480702064206C00F48050C5
:100F200018B9206C40F001002064204601F09AF8C6
:100F30000BE0206C00F0100018B1204601F094F88E
:100F400003E0A06BC16C2846884770BD70B50546AC
:100F5000AC6B40202064606C40F00400606420466C
:100F600001F082F870BD70B50446A56B284601F00B
:100F70007AF870BD55494A6822F440324A604A689E
:100F800043681A434A600268526822F48072036818
:100F90005A6002685368026943EA022203685A6091
:100FA0000268526822F0407203685A600268526810
:100FB00083681A4303685A600268926822F40062E8
:100FC00003689A6002689268C3681A4303689A606B
:100FD0003F4B826A9A4218D00268926822F070628F
:100FE00003689A6002689268836A1A4303689A6089
:100FF0000268926822F0405203689A600268926820
:10100000C36A1A4303689A600BE00268926822F090
:10101000706203689A600268926822F04052036826
:101020009A600268926822F0020203689A6002687D
:101030009368027E43EA420203689A602022125CAF
:10104000A2B10268526842F4006203685A60026802
:10105000526822F4604203685A6002685368426A28
:10106000521E43EA423203685A6005E00268526841
:1010700022F4006203685A600268D26A22F47002A5
:101080000368DA620268D36A828B521E43EA025214
:101090000368DA620268926822F4007203689A6058
:1010A0000268936890F8302043EA422203689A600D
:1010B0000268926822F4806203689A60026893680A
:1010C000426943EA822203689A6070470023014024
:1010D0000100000F10B505F0C1F8012211491248B6
:1010E00003F014FB04F0E4FD10EE104A2046FFF775
:1010F00057FB0E4A03C20D4890ED000B51EC100B4C
:10110000FFF77AFB00EE100A094880ED010A9FED17
:10111000090A094880ED000A9FED060A074880ED9C
:10112000000A10BD0C000020A0040020C80100200F
:101130002C0E002000000000D0010020D40100206F
:1011400000BFFEE710B501F09DFC0446154800689D
:10115000201A4EF66021884222D312480460802172
:101160001148FFF767F800201049088010A003F02D
:1011700077FE642001F06AFB11A10B48FFF765F8C8
:1011800058B91348007803280ADA11480078401C3F
:101190000F49087003F014FF02E000200C490870AA
:1011A00010BD000058000020EC0500205000002079
:1011B00041542B514D54434F4E4E3F0D0A000000F9
:1011C0002B514D54434F4E4E3A20302C33000000EB
:1011D0005C00002010B505F049FA0446124800787A
:1011E000844206D011480078401C104908700E480F
:1011F00004700F480068401C0D49086008460068EC
:1012000064280FD309480078052803DB0120094929
:10121000087002E0022007490870002003490870A6
:101220000349086010BD00001102002012020020D6
:1012300014020020100200200448408803498988D5
:10124000884201DD012070470020FCE710000020EB
:1012500070B50446012C08D10020134908701349C9
:1012600008700120124908701CE0DCB90020104908
:10127000087010480578002000F0D8F8002000F031
:101280002DF8002000F03CF8002000F069F8002064
:1012900005F040F801200449087004490870054829
:1012A000057000BF70BD000048000020490000200C
:1012B000810000202C01002010B504462CB1012231
:1012C0001021054801F0D8FB04E00022102102485B
:1012D00001F0D2FB10BD00000018024010B504461A
:1012E0002CB101220421054801F0C6FB04E00022D4
:1012F0000421024801F0C0FB10BD000000180240AC
:1013000010B504462CB101220821054801F0B4FBB8
:1013100004E000220821024801F0AEFB10BD0000ED
:101320000018024010B5044684B10C48007830B96A
:101330000120FFF7D3FF0020FFF7E2FF0CE00020C1
:10134000FFF7CCFF0120FFF7DBFF05E00020FFF7F0
:10135000C5FF0020FFF7D4FF10BD000038010020BA
:1013600010B504460CB1012000E0002002464FF405
:101370000071024801F080FB10BD0000001802401F
:1013800010B5044684B10C48007830B1012000F05B
:1013900029F8002000F038F80CE0002000F022F8D6
:1013A000012000F031F805E0002000F01BF80020DB
:1013B00000F02AF810BD00000002002010B5084817
:1013C000007830B1012000F00DF8002000F01CF88A
:1013D00005E0002000F006F8012000F015F810BD2F
:1013E0000002002010B504460CB1012000E00020EE
:1013F00002460421024801F03FFB0248447210BD3E
:10140000001002406C09002010B504460CB1012008
:1014100000E0002002460821024801F02DFB0248AE
:10142000847210BD001002406C09002010B5044603
:101430002CB101220221054801F01EFB04E000222C
:101440000221024801F018FB10BD00000018024004
:1014500010B5024801F01AF810BD00007805002010
:101460000146087810381823B0FBF3F20848805C76
:10147000C865032A05D908686FF30900001D88654F
:1014800003E008686FF309008865886D7047000005
:10149000D08A0008014600208A6A8B69CBB932B134
:1014A000012A0DD0022A03D0032A10D10EE000BF7A
:1014B000CB6A03F08073B3F1807F00D1012007E095
:1014C000CB6AB3F1C07F00D1012001E000E000BF92
:1014D00034E08B69B3F5005F1AD132B1012A07D02D
:1014E000022A03D0032A11D10AE000BF01200EE036
:1014F000CB6A03F08073B3F1807F00D1012006E056
:10150000CB6AB3F1C07F00D1012000E000BF15E03D
:1015100032B1012A05D0022A04D0032A0CD103E0FB
:1015200000BF00BF012008E0CB6A03F08073B3F175
:10153000807F00D1012000E000BF00BF704730B5C0
:101540000468246824F4802405682C6004686360BF
:101550008468402C04D10468A2600468E16003E060
:101560000468A1600468E26030BD00002DE9F04F1E
:101570002DED0A8B83B001F085FA0446D748006848
:10158000201AB0F57A7F07D20020D549088003B031
:10159000BDEC0A8BBDE8F08FD148008800F4004014
:1015A00000287CD04FF0000B0026002002908146DE
:1015B00000258246019000900027022004E0C949DE
:1015C000095C0F44411CC8B21728F8DBF8B2C549C2
:1015D000C97D88427DD1C34880780104C148C07864
:1015E00001EB0020BF49097900EB010BBD484079B0
:1015F0000104BC48807901EB0020BA49C97946183A
:1016000076B1BBFBF6F84046FFF7A4F841EC180BA7
:101610009FEDB50B53EC102BFEF7BBFFB44A03C292
:10162000B048007A0104AF48407A01EB0020AD4990
:10163000897A08440290AB48C07A0104A948007B2B
:1016400001EB0020A749497B00EB0109B9F1000F2C
:101650001FD04846FFF77EF841EC190B0298FFF7C0
:1016600079F841EC1B0B9FEDA30B53EC102BFEF70D
:1016700090FF41EC1A0B53EC192BFEF7FCFF41ECE9
:10168000180B9FED9C0B53EC102BFEF7F4FF9B4ABD
:1016900003C29448807B01049248C07B00E015E1BE
:1016A00001EB00208F49097C45188E48407C0104DD
:1016B0008C48807C01EB00208A49C97C00EB010A40
:1016C000BAF1000F10D0B5FBFAF84046FFF742F828
:1016D00000E0B1E041EC180B9FED830B53EC102BB5
:1016E000FEF757FF864A03C27E48007D00F0800067
:1016F0008449098888420AD083480078401C82497E
:1017000008707848007D00F080007E4908807E489F
:10171000007801047348407D01EB00207149897D08
:10172000084401909FED790B53EC102B744890ED19
:10173000000B51EC100BFFF747F87DD8002D7BD044
:101740002846FFF707F841EC1B0B9FED670B53ECA6
:10175000102BFEF71EFF41EC1A0B53EC1A2B9FEDDA
:101760006D0B51EC100BFEF786FF41EC190B9FED52
:101770006B0B53EC102BFEF70CFF41EC180BFEF734
:10178000F6FF00900098FEF7E5FF41EC1A0B019878
:10179000FEF7E0FF41EC1C0B9FED600B53EC102BB0
:1017A000FEF7F7FE41EC1B0B53EC1A2BFEF763FF21
:1017B00041EC190B9FED590B53EC102BFEF75BFF1F
:1017C00041EC180BFFF718F85649086001F05AF978
:1017D000804655480068A8EB00004EF6602188421C
:1017E00072D3504890ED000A5048D0ED000A30EE18
:1017F000600AB0EE408AB5EEC08AF1EE10FA59DD0B
:10180000B7EE000AB4EEC08AF1EE10FA52D218EE2A
:10181000100AFEF7C5FF41EC190B454890ED000B8F
:1018200053EC102B51EC190BFEF70CFE404A03C28F
:101830003F4890ED000B00E047E051EC100BFEF745
:10184000DBFF00EE100A3B4880ED010A3A480068D1
:10185000FEF780FF41EC1A0B354890ED000B53EC7E
:10186000102B51EC1A0BFEF791FE41EC190B9FED7A
:10187000330B53EC102BFEF7A7FF05D93148006856
:10188000201A3149884215D9294890ED000B51ECB6
:10189000100BFEF7B1FF08EE900AB0EE680A04F0F4
:1018A00052FF234890ED000B51EC100BFEF75FFF49
:1018B000214908601B4890ED000A1C4880ED000A91
:1018C0001948C0F8008000BF00BF00BF0348046093
:1018D00000200349088000BF59E60000D80100201D
:1018E000940100207C09002014AE47E17A14FE3FE9
:1018F000A80100200000000000005940B0010020B5
:10190000B80100209E0100209D0100200000000081
:1019100000000000000000002A75B5410000000032
:101920000088C340D4010020E4010020D001002041
:10193000C80100202C0E0020E0010020000000A0C3
:101940009999B93FDC010020E09304007047000042
:1019500010B503F0D7FA05F099FA0020FFF766FDFD
:101960000020FFF7BBFC0020FFF7CAFC00200A495B
:1019700008600A4908600A4908700120094908708E
:1019800000200949087004F02BFE08490870084639
:1019900000780749087010BD300100203401002094
:1019A00038010020390100203A0100203B010020CD
:1019B0003C01002010B504F01BFE04465C48007892
:1019C000844209D000205B4908605B49086001201F
:1019D0005A49087056480470002C52D15848007873
:1019E00030B10020FFF722FD0020564908601FE0BB
:1019F0005048006854490968884206D20120FFF720
:101A000015FD01204F49086012E04F4800684F491A
:101A10000968084447490968884206D90020FFF749
:101A200005FD00204749086002E0002041490860A8
:101A30004748007818B10020FFF774FC77E03E4873
:101A4000006844490968884203D20120FFF76AFC14
:101A50006DE00020FFF766FC3E4800683E490968DB
:101A6000084435490968884261D800203249086035
:101A70003A48007808B9012000E000203749087092
:101A800055E00020FFF7D2FC00202E4908603048C6
:101A9000007818B10020FFF745FC48E0274800789F
:101AA00020B3254800682E490968884203D20120E6
:101AB000FFF738FC3BE00020FFF734FC28480068C3
:101AC0002849096808441C49096888422FD8002021
:101AD000194908602148007808B9012000E0002079
:101AE0001E49087000201549087020E0124800685F
:101AF0001D490968884203D20120FFF713FC16E054
:101B00000020FFF70FFC18480068184909680844CE
:101B10000949096888420AD80020074908600F4827
:101B2000007808B9012000E000200C49087010BDC1
:101B30004401002030010020340100203901002040
:101B40004800002040010020A8000020AC00002038
:101B500049000020B0000020B4000020380100201F
:101B6000C0000020C4000020B8000020BC000020FD
:101B700010B50E48007858B10D480068052807D305
:101B80000020FFF799FB0020084908700849086009
:101B900008480068482808D300200649086001204A
:101BA000FFF78AFB01200149087010BD30020020B8
:101BB000280200202C02002072B600BFFEE70000C1
:101BC00010B504F015FD04465E480078844209D043
:101BD00000205D4908605D49086001205C4908708B
:101BE00058480470002C53D15A48007830B1002076
:101BF000FFF71CFC0020584908601FE052480068AD
:101C000056490968884206D20120FFF70FFC0120DF
:101C10005149086012E05148006851490968084478
:101C200049490968884206D90020FFF7FFFB0020D8
:101C30004949086002E000204349086049480078AB
:101C400018B10020FFF76EFB7AE040480068464973
:101C50000968884203D20120FFF764FB70E0424824
:101C6000006842490968084438490968884203D92C
:101C70000020FFF757FB63E00020344908603C4830
:101C8000007808B9012000E000203949087057E0C9
:101C90000020FFF7CBFB00202F4908603148007877
:101CA00018B10020FFF73EFB4AE02948007828B32E
:101CB000264800682F490968884203D20120FFF7AF
:101CC00031FB3DE02B4800682B49096808441F4957
:101CD0000968884203D90020FFF724FB30E0002088
:101CE0001A4908602248007808B9012000E0002065
:101CF0001F49087000201649087021E01348006849
:101D00001E490968884203D20120FFF70BFB17E048
:101D10001A4800681A49096808440C490968884249
:101D200003D90020FFF7FEFA0AE000200749086007
:101D30000F48007808B9012000E000200C49087025
:101D400010BD0000460100203001002034010020B9
:101D5000390100204800002040010020C800002078
:101D6000CC00002049000020D0000020D40000203A
:101D700038010020E0000020E4000020D80000200E
:101D8000DC00002010B580211048FEF753FA002037
:101D90000F4908800FA003F063F8642000F056FD9F
:101DA0000FA10A48FEF751FA04466CB1083400E06E
:101DB000641C20782028FBD0132221460A48FEF715
:101DC00056FA00200849C87410BD0000EC05002038
:101DD0005000002041542B51434349440D0A000058
:101DE0002B51434349443A00D805002010B50B4815
:101DF0000078012804D10AA005F05AFE012010BD88
:101E0000FFF71AFA20B10DA005F052FE0220F6E706
:101E100012A005F04DFE0020F1E7000010020020A6
:101E2000E5BD93E5898DE4BDBFE794A8E5B882E7F9
:101E300094B5E4BE9BE794B50D0A0000E5BD93E5BB
:101E4000898DE4BDBFE794A8E5A4AAE998B3E88327
:101E5000BDE4BE9BE794B55C720A0000E5BD93E566
:101E6000898DE697A0E4BE9BE794B55C720A0000FA
:101E700038B580210D48FEF7DDF900200C490880B7
:101E80000CA002F0EDFF0EA10848FEF7DEF90446B3
:101E90005CB16A460CA12046FEF712FA012803D174
:101EA000009840B20B49087000BF38BDEC05002017
:101EB0005000002041542B4353510D0A00000000F4
:101EC0002B4353513A0000002B4353513A202564D1
:101ED000000000005500002038B5024600200090A8
:101EE00000BF92F83C00012801D1022038BD01203A
:101EF00082F83C0000BF0868092816D91068C0683D
:101F00000C780A3C04EB44050724AC40A043146859
:101F1000E0600C780A3C04EB44048868A040146834
:101F2000E46820431468E06013E0106800690C78EE
:101F300004EB44050724AC40A043146820610C78EE
:101F400004EB44048868A0401468246920431468A2
:101F500020614868072817D21068406B0C79641E0E
:101F600004EB84051F24AC40A04314686063088818
:101F700080B20C79641E04EB8404A0401468646B86
:101F800020431468606331E048680D2817D2106858
:101F9000006B0C79E41F04EB84051F24AC40A043C4
:101FA00014682063088880B20C79E41F04EB840471
:101FB000A0401468246B20431468206316E0106866
:101FC000C06A0C790D3C04EB84051F24AC40A0438F
:101FD0001468E062088880B20C790D3C04EB84043C
:101FE000A0401468E46A20431468E062194B1A4C5C
:101FF0001068A04206D10868122803D1586840F43E
:1020000080005860144C1068A0421CD10868102849
:1020100002D00868112816D1586840F400005860B2
:10202000086810280FD10D4800680D4CB0FBF4F083
:1020300000EB80004000009002E00098401E0090FD
:1020400000980028F9D100BF002082F83C0000BFB2
:1020500000BF4BE700230140002001403800002072
:1020600040420F00704770477047000070B504464B
:1020700000250CB9012070BD1549A06A884200D026
:1020800000BF206C30B9204600F024F800206064C6
:1020900084F83C00206C00F0100088B9206C20F41B
:1020A000885040F0020020642046FEF763FF0020C5
:1020B0006064206C20F0020040F00100206400E029
:1020C000012500BF002084F83C0000BF2846D2E76D
:1020D0000100000F10B586B00446142101A8FEF7D8
:1020E000A9F84149206888422CD100BF0020009007
:1020F0003E48006840F480703C490860084600682B
:1021000000F48070009000BF00BF00BF002000906E
:1021100036481438006840F001003449143908602A
:102120000846006800F00100009000BF00BF0120D9
:102130000190032002900020039001A92C4800F098
:1021400099FB4FE02B49206888424BD100BF00200B
:1021500000902648006840F48060244908600846E2
:10216000006800F48060009000BF00BF00BF002046
:1021700000901E481438006840F020001B491439B4
:1021800008600846006800F02000009000BF00BF13
:102190004FF4AC700190032002900020039001A93D
:1021A000154800F067FB1548154908608005486030
:1021B000002113488160C1604FF4806101614900D2
:1021C0004161890081614911C1610021016241625F
:1021D00000F07CFA08B1FFF7EFFC00BF0848A063ED
:1021E000846300BF06B010BD0020014044380240A7
:1021F000000002400022014000140240106402402E
:10220000CC020020F8B504460D461646002000908A
:1022100000BF94F83C00012801D10220F8BD012044
:1022200084F83C0000BF2068806800F00100A0B97D
:102230002068806840F00100216888605548006887
:102240005549B0FBF1F000EB4000009002E000982F
:10225000401E009000980028F9D12068806800F4A2
:102260008070B0F5807F05D12068806820F4807090
:10227000216888602068806800F0010000287ED016
:10228000206C40F20161884340F480702064206833
:10229000406800F4806028B1206C20F4005040F4C5
:1022A00080502064206C00F48050B0F5805F04D131
:1022B000606C20F00600606401E00020606400BFF4
:1022C000002084F83C0000BF344F3548A16BC86340
:1022D0003448A16B08643448A16BC8646FF02200D5
:1022E000216808602068406840F08060216848608C
:1022F0002068806840F4807021688860226802F15C
:102300004C0133462A46A06B00F056FA786800F07C
:102310001F0018BB25492068884213D02449206833
:10232000884204D1381D006800F01F0050B12149D7
:10233000206888422BD11948001D006800F01F005A
:10234000102824D22068806800F04050F8B9206836
:10235000806840F080402168886018E01349206858
:10236000884214D12068806800F0405078B9206815
:10237000806840F080402168886008E0FFE7206CBA
:1023800040F010002064606C40F0010060640020A8
:1023900044E700003800002040420F0000230140C5
:1023A000CF0E0008670F00084D0F00080020014005
:1023B000002101400022014070B50446A56D00F0E7
:1023C00061FB064694F83500022808D0802060653D
:1023D00000BF002084F8340000BF012070BD2068D9
:1023E000006820F01600216808602068406920F02D
:1023F000800021684861206C08B9A06C28B1206871
:10240000006820F00800216808602068006820F05B
:1024100001002168086010E000F034FB801B0528F3
:102420000BD920206065032084F8350000BF002010
:1024300084F8340000BF0320D0E72068006800F073
:1024400001000028E8D194F85C103F208840A86083
:10245000012084F8350000BF002084F8340000BF5C
:1024600000BFBBE7014691F83500022803D0802069
:10247000486501207047052081F83500086800682C
:1024800020F001000A6810600020F3E7F8B5044668
:10249000002000908C4800684FF41651B0FBF1F713
:1024A000A56D2E6894F85C1008208840304098B1E3
:1024B0002068006800F0040070B12068006820F017
:1024C00004002168086094F85C1008208840A86027
:1024D000606D40F00100606594F85C100120884058
:1024E000304068B12068406900F0800040B194F845
:1024F0005C1001208840A860606D40F002006065BB
:1025000094F85C1004208840304068B1206800686E
:1025100000F0020040B194F85C1004208840A860EC
:10252000606D40F00400606594F85C1010208840F5
:10253000304078B32068006800F0080050B394F889
:102540005C1010208840A8602068006800F480209B
:1025500080B12068006800F4002028B9206CC8B160
:102560002046216C884715E0A06C98B12046A16CEC
:1025700088470FE02068006800F4807028B9206860
:10258000006820F0080021680860206C10B1204627
:10259000216C884794F85C10202088403040002847
:1025A00065D02068006800F0100000285FD094F823
:1025B0005C1020208840A86094F83500052828D1B8
:1025C0002068006820F016002168086020684069D3
:1025D00020F0800021684861206C08B9A06C28B107
:1025E0002068006820F008002168086094F85C10FA
:1025F0003F208840A860012084F8350000BF0020FB
:1026000084F8340000BF206D10B12046216D88474A
:10261000F8BD2068006800F4802080B12068006860
:1026200000F4002028B9606C10B12046616C884726
:102630001DE0E06BD8B12046E16B884717E02068C9
:10264000006800F4807068B92068006820F010000D
:1026500021680860012084F8350000BF002084F85C
:10266000340000BFE06B10B12046E16B8847606D1D
:1026700038B3606D00F00100F0B1052084F835003A
:102680002068006820F001002168086000BF009801
:10269000401C0090B84200D905E02068006800F0B6
:1026A00001000028F3D100BF012084F8350000BFED
:1026B000002084F8340000BFE06C10B12046E16CCB
:1026C000884700BFA4E70000380000202DE9F04152
:1026D0000446002500F0D6F9074614B90120BDE8EC
:1026E000F081606A00B100BF022084F8350000BFAD
:1026F000002084F8340000BF2068006820F001004A
:10270000216808600AE000F0BDF9C01B052805D962
:1027100020206065032084F83500E0E72068006829
:1027200000F001000028EED120680568214805402E
:10273000D4E901010843E16808432169084361695C
:102740000843A1690843E1690843216A0843054336
:10275000606A042803D1D4E90B01084305432068CB
:1027600005602068456925F00705606A0543606AD1
:1027700004280DD1A06A0543E06A48B12046FEF75F
:1027800089FE28B140206065012084F83500A6E765
:10279000206845612046FEF763FE064694F85C100B
:1027A0003F208840B06000206065012084F835003B
:1027B000002094E73F8010F02DE9F04704460D46D5
:1027C00016461F464FF00008D4F8589000BF94F802
:1027D0003400012802D10220BDE8F087012084F8EE
:1027E000340000BF94F83500012825D1022084F878
:1027F0003500002060653B46324629462046FEF7FC
:102800009EFE94F85C103F208840C9F808002068BC
:10281000006840F0160021680860206C28B120682C
:10282000006840F00800216808602068006840F0F7
:1028300001002168086006E000BF002084F8340031
:1028400000BF4FF002084046C6E7000070B50446DE
:1028500000F018F906462546681C10B104480078B7
:10286000054400BF00F00EF9801BA842FAD370BDEA
:1028700034000020F8B502460B4600250024002055
:102880000021D6E0012606FA01F51E6806EA0504D5
:10289000AC4274D11E7906F00306012E04D01E79D5
:1028A00006F00306022E13D190684F000326BE40A7
:1028B000B0434F00DE68BE40304390605068012650
:1028C0008E40B0431E79C6F300168E4030435060F0
:1028D0001E7906F00306032E09D0D0684F000326A8
:1028E000BE40B0434F009E68BE403043D0601E796A
:1028F00006F00306022E13D1CF0802F1200656F887
:1029000027004E07F70E0F26BE40B0434F07FF0EBD
:102910001E69BE403043CF0802F1200646F827006A
:1029200010684F000326BE40B0431E7906F0030630
:102930004F00BE40304310605E6806F44036002E03
:1029400076D000BF002600963C4E366846F480469E
:102950003A4F3E603E46366806F48046009600BF19
:1029600000BF374E8F0856F827008E07370F0F2607
:10297000BE40B043334EB24202D1002624E057E0BD
:10298000314EB24201D101261EE0304EB24201D199
:10299000022619E02E4EB24201D1032614E02D4E3C
:1029A000B24201D104260FE02B4EB24201D10526DE
:1029B0000AE02A4EB24201D1062605E0284EB24274
:1029C00001D1072600E008268F073F0FBE403043A5
:1029D0001B4E8F0846F82700224E3068A0435E68E1
:1029E00006F4801606B120431E4E3060361D306856
:1029F000A0435E6806F4001606B12043194E361D4A
:102A00003060184E361F3068A0435E6806F400360A
:102A100006B12043134E361F3060361F3068A04386
:102A20005E6806F4803606B120430E4E083E3060E4
:102A3000491C1029FFF426AFF8BD000044380240BD
:102A40000838014000000240000402400008024033
:102A5000000C024000100240001402400018024026
:102A6000001C0240083C0140024613690B400BB1B8
:102A7000012000E0002070470AB1816101E00B04F1
:102A80008361704701480068704700002C000020F7
:102A900070B504460CB9012070BD94F83D0028B90A
:102AA000002084F83C00204600F010FB242084F82D
:102AB0003D002068006820F001002168086020685F
:102AC000006840F40040216808602068006820F435
:102AD00000402168086000F0DFFC05465C49606842
:102AE000884206D85B48854201D2012007E00020D9
:102AF00005E05948854201D2012000E0002001286C
:102B000000D1C9E75548B5FBF0F62068406820F0D1
:102B10003F003043216848604D496068884201D8D1
:102B2000701C07E04FF4967070434FF47A71B0FB5D
:102B3000F1F0401C2168096A21F03F010843216837
:102B4000086243496068884214D8681E6168490079
:102B5000B0FBF1F0401CC0F30B00042801D20420AC
:102B60003DE0681E61684900B0FBF1F0401CC0F315
:102B70000B0034E0A06838B9681E616801EB4101C0
:102B8000B0FBF1F0401C0AE0681E616801EBC10275
:102B900002EB0111B0FBF1F0401C40F48040C0F3A7
:102BA0000B0008B901201AE0A06848B9681E6168E6
:102BB00001EB4101B0FBF1F0401CC0F30B000CE055
:102BC000681E616801EBC10202EB0111B0FBF1F07C
:102BD000401CC0F30B0040F4804040F400402168EA
:102BE000C9694CF6FF72914308432168C861D4E972
:102BF000070108432168096821F0C00108432168E2
:102C00000860D4E9031008432168896848F2FF325C
:102C10009143084321688860D4E90501084321688D
:102C2000C96821F0FF0108432168C8602068006876
:102C300040F001002168086000202064202084F812
:102C40003D000020206384F83E0000BF24E7000020
:102C5000A086010080841E0000093D0040420F0054
:102C60002DE9FC5F04460F4690469946DDE90CAB22
:102C70000E9EFFF707FF054694F83D00202870D10F
:102C800019230122B5492046009501F06EFF10B1CD
:102C90000220BDE8FC9F00BF94F83C00012801D150
:102CA0000220F6E7012084F83C0000BF206800689D
:102CB00000F0010028B92068006840F00100216898
:102CC00008602068006820F4006021680860222005
:102CD00084F83D00402084F83E0000202064C4F8C1
:102CE00024A0A4F82AB0608D20859D48E0624B4660
:102CF000424639462046CDE9006501F0E3FD08B1C2
:102D00000120C6E7208D88B900BF0020019020680F
:102D10004069019020688069019000BF00BF206871
:102D2000006840F400702168086040E0208D0128B0
:102D300018D12068006820F480602168086000BF16
:102D4000002001902068406901902068806901900E
:102D500000BF00BF2068006840F400702168086070
:102D600025E0F8E0208D022816D12068006820F4C4
:102D70008060216808602068006840F40060216875
:102D8000086000BF00200190206840690190206821
:102D90008069019000BF0AE000BF00200190206818
:102DA0004069019020688069019000BF00BFC3E0C6
:102DB000208D03287ED8208D012815D12A46314642
:102DC000204601F0AEFF08B1012062E720680069EB
:102DD000616A0870606A401C6062208D401E208518
:102DE000608D401E6085A7E0208D02282AD13346E1
:102DF00000225C492046009501F0B7FE08B1012091
:102E000047E72068006840F4007021680860206887
:102E10000069616A0870606A401C6062208D401E13
:102E20002085608D401E608520680069616A087099
:102E3000606A401C6062208D401E2085608D401EAF
:102E4000608579E03346002246492046009501F02E
:102E50008CFE08B101201CE72068006820F4806027
:102E60002168086020680069616A0870606A401C17
:102E70006062208D401E2085608D401E6085334637
:102E8000002238492046009501F06FFE08B101206C
:102E9000FFE62068006840F4007021680860206840
:102EA0000069616A0870606A401C6062208D401E83
:102EB000208500E010E0608D401E6085206800697C
:102EC000616A0870606A401C6062208D401E208527
:102ED000608D401E60852FE02A463146204601F075
:102EE00020FF08B10120D4E620680069616A0870FB
:102EF000606A401C6062208D401E2085608D401EEF
:102F0000608520684069C0F38000A8B1208D032847
:102F100005D12068006820F480602168086020687E
:102F20000069616A0870606A401C6062208D401E02
:102F30002085608D401E6085208D00287FF438AF8D
:102F4000202084F83D00002084F83E0000BF84F873
:102F50003C0000BF9DE602209BE60000020010003E
:102F60000000FFFF040001002DE9FC5F04460F464E
:102F700090469946DDE90CAB0E9EFFF783FD0546B2
:102F800094F83D0020287DD1192301224D49204687
:102F9000009501F0EAFD10B10220BDE8FC9F00BFE2
:102FA00094F83C00012801D10220F6E7012084F8C2
:102FB0003C0000BF2068006800F0010028B92068CC
:102FC000006840F00100216808602068006820F473
:102FD000006021680860212084F83D00402084F8CA
:102FE0003E0000202064C4F824A0A4F82AB0608D1C
:102FF00020853548E0624B46424639462046CDE9B9
:10300000006501F00FFD08B10120C6E731E02A4656
:103010003146204601F0CAFE50B1206C042805D18B
:103020002068006840F40070216808600120B4E75F
:10303000606A007821680861606A401C6062208DC7
:10304000401E2085608D401E608520684069C0F369
:10305000800070B1208D60B1606A007821680861DD
:10306000606A401C6062208D401E2085608D401E7D
:103070006085208D0028CAD12A463146204601F0BD
:1030800041FD00E01CE050B1206C042805D120680F
:10309000006840F400702168086001207DE7206826
:1030A000006840F4007021680860202084F83D002A
:1030B000002084F83E0000BF84F83C0000BF6CE7AD
:1030C00002206AE7020010000000FFFF10B586B082
:1030D0000446142101A8FDF7ADF81B492068884279
:1030E0002FD100BF002000901848006840F0200059
:1030F000164908600846006800F02000009000BFF4
:1031000000BF0320019012200290002003900320B2
:1031100004900420059001A90D48FFF7ABFB00BF08
:103120000020009009481030006840F480000749F2
:10313000103108600846006800F48000009000BF6D
:1031400000BF06B010BD00000058004030380240FB
:103150000014024003480068034909780844014903
:10316000086070472C0000203400002010B50D4886
:10317000006840F400700B4908600846006840F49D
:10318000806008600846006840F480700860032092
:1031900000F0A6F80F2000F007F800F02BF8002050
:1031A00010BD0000003C024070B504460E48007897
:1031B0004FF47A71B1FBF0F00C490968B1FBF0F5FE
:1031C000284600F02FFC08B1012070BD102C07D25A
:1031D00000222146501E00F045F80548046001E039
:1031E0000120F2E70020F0E7340000203800002042
:1031F0003000002008B500BF002000900E48006895
:1032000040F480400C4908600846006800F48040A3
:10321000009000BF00BF00BF00200090081F0068A2
:1032200040F08050091F08600846006800F0805098
:10323000009000BF00BF08BD443802400146084668
:1032400000280DDB00BF00BF00F01F0301229A40E1
:1032500043099B0003F1E023C3F8002100BF00BF36
:1032600000BF70472DE9F05F80460D4616460027E7
:1032700004F042FC074639462A46334601F007006F
:10328000C0F1070ABAF1040F02D94FF0040A01E0B5
:10329000C0F1070AD14600F1040ABAF1070F02D2C1
:1032A0004FF0000A01E0A0F1030AD4464FF0010AF2
:1032B0000AFA09FAAAF1010A0AEA020A0AFA0CFA57
:1032C0004FF0010B0BFA0CFBABF1010B0BEA030BFC
:1032D0004AEA0B042146404604F016FCBDE8F09F84
:1032E00000BF00F00702064B19684FF6FF031940B4
:1032F000044B0B4343EA0221014B196000BF7047A6
:103300000CED00E00000FA0570B504460D460CB95E
:10331000012070BD5848006800F00700A84209D29B
:1033200055490D700846006800F00700A84201D01A
:103330000120EEE7207800F0020002281DD120785D
:1033400000F00400042805D14C48006840F4E05027
:103350004A490860207800F00800082805D147484D
:10336000006840F46040454908604448006820F027
:10337000F000A168084341490860207800F001008E
:10338000A8B36068012807D13C4808380068C0F33A
:103390004040B8B90120BCE76068022802D06068EC
:1033A000032807D1354808380068C0F3406048B9A1
:1033B0000120AEE7314808380068C0F3400008B982
:1033C0000120A6E72D48006820F00300616808434B
:1033D0002A490860FFF756FB064609E0FFF752FB53
:1033E000801B41F28831884202D9032091E707E02F
:1033F0002248006800F00C006168B0EB810FEDD14D
:103400001D48006800F00700A84209D91A490D704C
:103410000846006800F00700A84201D0012078E7C4
:10342000207800F00400042807D11448006820F434
:10343000E050E168084311490860207800F0080076
:10344000082808D10D48006820F46040216940EA4E
:10345000C1000A49086000F03FF808490968C1F353
:103460000311074A515CC8400649086006480068D5
:10347000FFF79AFE00204CE7003C0240083802406B
:10348000D88A000838000020300000200148006879
:10349000704700003800002000B5FFF7F7FF04492F
:1034A0000968C1F38221034A515CC84000BD000095
:1034B00008380240E88A000800B5FFF7E7FF044932
:1034C0000968C1F34231034A515CC84000BD0000A5
:1034D00008380240E88A00082DE9F047002400255A
:1034E0000026A1462548006800F00C0020B1042801
:1034F00005D008283AD105E0DFF8849039E0DFF8FC
:10350000849036E01D48001F006800F03F041B480F
:10351000001F006800F4800078B11A481749091F9D
:103520000968C1F38811A0FB0170014622460023FF
:103530003846FCF747FE05460EE011480F49091FC3
:103540000968C1F38811A0FB0170014622460023DF
:103550003846FCF737FE05460848001F0068C0F3F0
:103560000140401C4600B5FBF6F902E0DFF8109080
:1035700000BF00BF4846BDE8F087000008380240A1
:103580000024F40000127A00F8B504460CB90120BA
:10359000F8BD207800F00100002874D0F9480068D8
:1035A00000F00C0004280DD0F648006800F00C0074
:1035B000082813D1F348001F006800F48000B0F51C
:1035C000800F0BD1EF4808380068C0F34040002856
:1035D00059D06068002856D10120D9E700BF606843
:1035E000B0F5803F08D1E7480838006840F48030E3
:1035F000E449083908601EE06068B0F5A02F0DD1DD
:10360000E0480838006840F48020DE490839086046
:103610000846006840F4803008600CE0D94808385B
:10362000006820F48030D7490839086008460068EF
:1036300020F48020086000BF606890B1FFF722FA94
:10364000054606E0FFF71EFA401B642801D9032057
:103650009EE7CC4808380068C0F340400028F1D00D
:1036600011E0FFF70FFA054606E0FFF70BFA401BE3
:10367000642801D903208BE7C24808380068C0F3EA
:1036800040400028F1D1207800F0020002285FD1EC
:10369000BC48006800F00C0058B1BA48006800F05F
:1036A0000C0008281CD1B748001F006800F48000F7
:1036B000B0B9B44808380068C0F3400020B1E068F1
:1036C000012801D0012063E7AE480838006820F0E7
:1036D000F800216940EAC100AA490839086037E0CA
:1036E000E06800B30120A8490860FFF7CBF9054660
:1036F00006E0FFF7C7F9401B022801D9032047E77E
:10370000A04808380068C0F340000028F1D09D4868
:103710000838006820F0F800216940EAC1009949A2
:103720000839086014E0002097490860FFF7AAF9FB
:10373000054606E0FFF7A6F9401B022801D9032041
:1037400026E7904808380068C0F340000028F1D10F
:10375000207800F0080008282CD16069A8B1012069
:103760008A490860FFF78EF9054606E0FFF78AF9F7
:10377000401B022801D903200AE782486C30006808
:10378000C0F340000028F1D014E000207F49086019
:10379000FFF778F9054606E0FFF774F9401B0228A9
:1037A00001D90320F4E677486C300068C0F340008C
:1037B0000028F1D1207800F00400042870D10027FF
:1037C00070483830006800F0805090B900BF002089
:1037D00000906C483830006840F0805069493831BA
:1037E00008600846006800F08050009000BF00BFED
:1037F00001276748006800F48070B0B96448006829
:1038000040F4807062490860FFF73CF9054606E025
:10381000FFF738F9401B022801D90320B8E65C48BD
:10382000006800F480700028F2D000BFA068012872
:1038300008D154486830006840F0010051496831AF
:1038400008601DE0A06805280DD14E48683000686A
:1038500040F004004B49683108600846006840F0B9
:10386000010008600CE047486830006820F0010063
:103870004449683108600846006820F00400086088
:1038800000BFA068A8B1FFF7FDF8054609E0FFF703
:10389000F9F8401B41F28831884202D9032077E6CB
:1038A00026E0384868300068C0F340000028EED0B9
:1038B00013E0FFF7E7F8054608E0FFF7E3F8401BE1
:1038C00041F28831884201D9032061E62D486830F1
:1038D0000068C0F340000028EFD1012F07D129482C
:1038E0003830006820F0805026493831086000BF29
:1038F000A069002845D02348006800F00C00082883
:103900005DD0A069022845D100201F490866FFF755
:10391000B9F8054606E0FFF7B5F8401B022801D9C3
:10392000032035E6174808380068C0F340600028D7
:10393000F1D1D4E907010843616A40EA811101220B
:10394000A06AC2EB500041EA00412C20005D41EA30
:1039500000600C49091F086001200B490866FFF749
:1039600091F8054606E0FFF78DF8401B022801D9C3
:1039700003200DE6034808380068C0F340600028C3
:10398000F1D049E00838024000004742800E47422B
:1039900000700040002021490866FFF773F80546D3
:1039A00006E0FFF76FF8401B022801D90320EFE57E
:1039B0001B480068C0F340600028F2D12CE0A069E9
:1039C000012800D1E4E51648001D0668A069012819
:1039D00020D006F48001E06981421BD106F03F014E
:1039E000206A814216D147F6C0703040616AB0EB60
:1039F000811F0FD106F440310122A06AC2EB5000B2
:103A0000B1EB004F06D106F070612C20005DB1EBE8
:103A1000006F01D00120BBE50020B9E5000047425E
:103A20000038024070B504462546681EB0F1807F1C
:103A300001D301200FE0681E4FF0E02148610F2103
:103A40004FF0FF3004F060F800204FF0E021886173
:103A500007200861002070BD7047704730B50246EE
:103A60000B4600BF92F83C00012801D1022030BD76
:103A7000012082F83C0000BF022082F83D0010685F
:103A800044681068816824F0700418680443106862
:103A90004460184D1068A8421BD01068B0F1804FE8
:103AA00017D0154D1068A84213D0144D1068A842C5
:103AB0000FD0134D1068A8420BD0124D1068A842C9
:103AC00007D0114D1068A84203D0104D1068A842CD
:103AD00005D121F080015868014310688160012000
:103AE00082F83D0000BF002082F83C0000BF00BF0C
:103AF000BDE7000000000140000400400008004055
:103B0000000C00400004014000400140001800404B
:103B100010B504460CB9012010BD94F83D0028B939
:103B2000002084F83C00204600F026F8022084F8AB
:103B30003D00211D206803F0F9F8012084F84600BB
:103B400000BF84F83E0001213F200155402001556F
:103B50004120015500BF00BF012084F842004320EE
:103B60000155442001554520015500BF012084F82E
:103B70003D000020D0E7000038B504462068B0F1D1
:103B8000804F18D100BF002000903648006840F0F8
:103B90000100344908600846006800F00100009008
:103BA00000BF00BF002203211C20FFF75BFB1C208D
:103BB000FFF744FB55E02C492068884218D100BF2C
:103BC000002000902748006840F002002549086066
:103BD0000846006800F00200009000BF00BF00220D
:103BE00011461D20FFF73EFB1D20FFF727FB38E0A5
:103BF0001E492068884218D100BF00200090194853
:103C0000006840F01000174908600846006800F09E
:103C10001000009000BF00BF002211463620FFF7C1
:103C200021FB3620FFF70AFB1BE011492068884280
:103C300017D100BF002000900A48006840F0200023
:103C4000084908600846006800F02000009000BFA6
:103C500000BF002211463720FFF704FB3720FFF793
:103C6000EDFA38BD4038024000040040001000402A
:103C700000140040014691F83D00012801D00120C8
:103C80007047022081F83D000868C06840F00100DC
:103C90000B68D8601A4B086898421BD00868B0F1CE
:103CA000804F17D0174B0868984213D0164B0868FE
:103CB00098420FD0154B086898420BD0144B0868F7
:103CC000984207D0134B0868984203D0124B0868FB
:103CD00098420CD10868806800F00702062A0CD0D0
:103CE0000868006840F001000B68186005E008688B
:103CF000006840F001000B6818600020C0E7000079
:103D0000000001400004004000080040000C00409A
:103D100000040140004001400018004001460868CE
:103D2000C06820F001000A68D06000BF0868006A1F
:103D300041F21112104050B90868006A9210104008
:103D400028B90868006820F001000A68106000BF08
:103D5000012081F83D00002070472DE9F041044624
:103D60000D46002700BF94F83C00012802D1022034
:103D7000BDE8F081012084F83C0000BF022084F8F7
:103D80003D002068866826F0770626F47F46206886
:103D900086602868502833D00CDC202850D004DC02
:103DA00000284BD0102851D149E0302849D0402874
:103DB0004CD139E060282DD0702807D0B0F5805F55
:103DC00003D0B0F5005F41D10DE041E0D5E9021329
:103DD0006A68206803F01EF82068866846F0770657
:103DE0002068866034E0D5E902136A68206803F031
:103DF00011F82068806840F480402168886027E0DE
:103E0000EA686968206803F019F85021206803F017
:103E10000CF81DE0EA686968206803F022F8602168
:103E2000206803F002F813E0EA686968206803F08C
:103E300005F84021206802F0F8FF09E000BF00BF4C
:103E400000BF2968206802F0F0FF01E0012700BFF1
:103E500000BF012084F83D0000BF002084F83C0032
:103E600000BF384684E7704770B504462068C568CF
:103E70002068066906F00200022819D105F0020048
:103E8000022815D1401F2168086101202077206891
:103E9000806900F0030018B12046FFF7E4FF05E059
:103EA000204600F097F8204600F095F80020207793
:103EB00006F00400042819D105F00400042815D1E7
:103EC000C04321680861022020772068806900F4DF
:103ED000407018B12046FFF7C6FF05E0204600F00D
:103EE00079F8204600F077F80020207706F00800E7
:103EF000082819D105F00800082815D1C043216809
:103F00000861042020772068C06900F0030018B120
:103F10002046FFF7A8FF05E0204600F05BF82046AA
:103F200000F059F80020207706F01000102819D171
:103F300005F01000102815D1C04321680861082041
:103F400020772068C06900F4407018B12046FFF760
:103F50008AFF05E0204600F03DF8204600F03BF8DF
:103F60000020207706F0010048B105F0010030B1D3
:103F70006FF0010021680861204600F02DF806F07E
:103F80008000802809D105F08000802805D1C04339
:103F9000216808612046FFF75FFD06F040004028D9
:103FA00009D105F04000402805D1C04321680861CF
:103FB000204600F09DF806F02000202809D105F0E9
:103FC0002000202805D1C043216808612046FFF762
:103FD00044FD70BD7047704710B5044635492068F0
:103FE000884211D134480088401C33490880084673
:103FF000008841F2883188425ADB00202E4908802F
:1040000001202E49087053E02068B0F1804F18D18C
:104010002B480068401C2A4908602A480068401C58
:104020002849086028480078042841D127480068BA
:10403000401C2649086026480068401C2449086046
:1040400036E024492068884219D123480068401C82
:10405000214908603C282BD3002008601F480068D5
:10406000401C1E4908603C2806D3002008601C48FC
:104070000068401C1A490860FDF77AFD18E01949EC
:104080002068884214D118480078401C16490870EE
:10409000084600783C280BDB02F04EF91348006814
:1040A000401C1249086002F091F900200E49087086
:1040B00010BD000000100040180000205400002037
:1040C00030010020340100202C01002024010020B8
:1040D00028010020001400402402002028020020B3
:1040E0002C0200200004004016000020F4010020F3
:1040F0007047F8B504460E46174694F8420020284B
:104100002ED106B10FB90120F8BD01202063002097
:1041100060633A463146204603F06AFA0546EDB937
:10412000206B012819D100BF002000902068006892
:10413000009020684068009000BF00BF00BF00BF33
:1041400021680C3151E8001F41F0100021680C314A
:1041500041E80002002AF3D100E001252846D3E718
:104160000220D1E770B505460C460649286888420A
:1041700006D1054804800A1504490548FFF7B9FF30
:1041800070BD00000044004050000020EC050020FD
:1041900030050020704700002DE9F84F04462068E4
:1041A00005682068C668206847694FF00009CA465C
:1041B00005F00F09B9F1000F0AD105F0200038B160
:1041C00006F0200020B1204603F07EF8BDE8F88F0D
:1041D000B9F1000F7CD007F0010018B906F4907017
:1041E000002875D005F0010030B106F4807018B1D8
:1041F000606C40F00100606405F0040030B107F02D
:10420000010018B1606C40F00200606405F002002B
:1042100030B107F0010018B1606C40F00400606438
:1042200005F0080048B106F0200010B907F00100C1
:1042300018B1606C40F008006064606C002846D0E3
:1042400005F0200028B106F0200010B1204603F050
:104250003BF820684069C0F3801A606C00F00800E9
:1042600010B9BAF1000F2DD0204602F0E7FF206808
:10427000406900F04000402820D100BF00BF216805
:10428000143151E8001F21F040002168143141E849
:104290000002002AF3D100BFE06B50B17748E16B18
:1042A0000865E06BFEF7DEF888B1E06B016D8847CA
:1042B0000DE02046FFF76EFF09E009E02046FFF71A
:1042C00069FF04E02046FFF765FF002060647DE79A
:1042D000206B012878D105F01000002874D006F07A
:1042E00010000028FAD000BF00200090206800686D
:1042F000009020684068009000BF00BF20684069BF
:1043000000F04000402860D1E06B006840681FFA70
:1043100080F8B8F1000F56D0A08D404553DDA4F8C9
:104320002E80E06BC069B0F5807F43D000BF00BF36
:1043300021680C3151E8001F21F4807021680C3194
:1043400041E80002002AF3D100BF00BF00BF21688E
:10435000143151E8001F21F001002168143141E8B7
:104360000002002AF3D100BF00BF00BF2168143152
:1043700051E8001F21F040002168143141E800029B
:10438000002AF3D100BF202084F8420000202063DF
:1043900000BF00BF21680C3151E8001F21F0100060
:1043A00021680C3141E80002002AF3D100BFE06B24
:1043B000FEF702F802206063A08DE28D801A81B2C0
:1043C0002046FFF7CFFE01E742E0A08DE18D401AC5
:1043D0001FFA80F8E08DD0B3B8F1000F37D000BFDE
:1043E00000BF21680C3151E8001F21F49070216852
:1043F0000C3141E80002002AF3D100BF00BF00BF2A
:104400002168143151E8001F21F0010021681431A6
:1044100041E80002002AF3D100BF202084F84200C6
:104420000020206300BF00BF21680C3151E8001F4D
:1044300021F0100021680C3141E80002002AF3D17C
:1044400000BF0220606341462046FFF78BFEBDE6B9
:1044500005F0800030B106F0800018B1204603F06E
:10446000E7F8B3E605F0400030B106F0400018B1BF
:10447000204602F019FFA9E600BFA7E6297200084E
:1044800010B504460CB9012010BDA06900B100E0D0
:1044900000BF94F8410028B9002084F8400020466D
:1044A00000F02AF8242084F841002068C06820F435
:1044B00000502168C860204602F084FF206800692F
:1044C00020F49040216808612068406920F02A00AB
:1044D000216848612068C06840F400502168C860C5
:1044E00000206064202084F8410084F8420000200D
:1044F000606300BFC8E7000010B586B00446142111
:1045000001A8FBF797FE78492068884275D100BF63
:10451000002000907548006840F40020734908604E
:104520000846006800F40020009000BF00BF00BFF4
:10453000002000906D481038006840F001006B4981
:10454000103908600846006800F00100009000BFC4
:1045500000BF00BF002000900846006840F0040043
:1045600008600846006800F00400009000BF00BF2B
:104570000220019002900020039003200490082064
:10458000059001A95A48FEF775F94FF48060019033
:104590000220029000200390032004900820059040
:1045A00001A95448FEF766F953485449086040058C
:1045B0004860002151488160C1604FF48061016111
:1045C0000021416181614FF48071C161002101626C
:1045D0004162FEF77BF808B1FDF7EEFA00BF4748ED
:1045E000E063846300BF002211463420FEF73AFEE8
:1045F0003420FEF723FE74E0FFE74149206888423B
:1046000033D100BF002000903848001D006840F002
:1046100010003649091D08600846006800F01000C7
:10462000009000BF00BF00BF002000902F4810384E
:10463000006840F001002D49103908600846006804
:1046400000F00100009000BF00BF4FF4C060019077
:104650000220029000200390032004900720059080
:1046600001A92348FEF706F93BE026492068884265
:1046700037D100BF002000901C48006840F4003093
:104680001A4908600846006800F40030009000BF36
:1046900000BF00BF0020009014481038006840F0B0
:1046A00008001249103908600846006800F0080048
:1046B000009000BF00BF6020019002200290002007
:1046C0000390032004900720059001A90E48FEF7EF
:1046D000D1F8002202212620FEF7C4FD2620FEF795
:1046E000ADFD06B010BD0000004C00404038024057
:1046F00000000240000802404060024078050020AF
:104700000010014000440040000C024070B5044617
:104710000D46164694F8420020280BD105B10EB97B
:10472000012070BD0020206332462946204602F059
:104730005FFFF6E70220F4E770B50446FEF7A2F942
:1047400005461949206888422CD118480088B0F5E0
:10475000167F1FDA16490A7814490888411C134B42
:10476000198014490A5418460088182815DB124885
:104770000068281AB0F57A7F08D31846008840F4FC
:104780000040194608800C48056006E000200749F3
:10479000088002E0002005490880012204490748FA
:1047A000FFF7B4FF70BD0000004C004094010020F2
:1047B0000C0000207C09002028000020A00400201C
:1047C0002DE9F84F04460E46174699464FF0000A69
:1047D00094F84100202850D106B117B90120BDE856
:1047E000F88F00206064212084F84100FEF74AF928
:1047F0008246A784E784A068B0F5805F04D1206971
:1048000010B90025B04602E035464FF000081EE022
:104810005346002280212046CDF8009002F038FF58
:1048200020B1202084F841000320D8E745B9B8F82A
:104830000000C0F308002168486008F1020803E0A6
:104840002878216848606D1CE08C401EE084E08C74
:104850000028DDD15346002240212046CDF80090AB
:1048600002F016FF20B1202084F841000320B6E7B3
:10487000202084F841000020B1E70220AFE7704714
:1048800000BFFEE7014608684069C0F38020B0B170
:104890006FF480600A68506100200863202081F86E
:1048A0003D00002081F83E00086C40F004000864E0
:1048B00000BF002081F83C0000BF012070470020AD
:1048C000FCE700002DE9F84304460F4615469946DB
:1048D000DDE908862068006840F48060216808608F
:1048E0002068006840F48070216808604346002218
:1048F0004FF001112046009600F037F960B12068B2
:10490000006800F48070B0F5807F02D14FF4007031
:1049100020640320BDE8F88307F0FE0021680861E9
:10492000334642463E49204600F07EF908B1012058
:10493000F0E700BF002000902068406900902068E8
:104940008069009000BF00BF32464146204600F01B
:104950002DFA50B1206C042805D12068006840F47D
:104960000070216808600120D4E7B9F1010F03D17C
:10497000E8B22168086117E0C5F3072021680861E3
:1049800032464146204600F011FA50B1206C04280E
:1049900005D12068006840F400702168086001209B
:1049A000B8E7E8B22168086132464146204600F087
:1049B000FDF950B1206C042805D12068006840F44E
:1049C0000070216808600120A4E72068006840F4B6
:1049D000807021680860434600224FF00111204694
:1049E000009600F0C2F858B12068006800F48070AA
:1049F000B0F5807F02D14FF400702064032089E776
:104A0000F8B240F00100216808613346424604498B
:104A1000204600F009F908B101207BE7002079E782
:104A2000020001002DE9F8430446884615469946E0
:104A3000DDE908672068006840F48070216808603C
:104A4000334600224FF001112046009700F08DF808
:104A500060B12068006800F48070B0F5807F02D1FA
:104A60004FF4007020640320BDE8F88308F0FE00D6
:104A7000216808613B4632462149204600F0D4F8BF
:104A800008B10120F0E700BF0020009020684069D5
:104A9000009020688069009000BF00BF3A46314610
:104AA000204600F083F950B1206C042805D120681D
:104AB000006840F40070216808600120D4E7B9F173
:104AC000010F03D1E8B22168086117E0C5F30720A0
:104AD000216808613A463146204600F067F950B136
:104AE000206C042805D12068006840F4007021681B
:104AF00008600120B8E7E8B2216808610020B3E748
:104B00000200010070B504460D46164625E0204619
:104B1000FFF7B8FE08B1012070BD681CE8B1FDF7D1
:104B2000B1FF801BA84200D8BDB920684069C0F31E
:104B3000800090B900202063202084F83D000020F0
:104B400084F83E00206C40F02000206400BF00206C
:104B500084F83C0000BF0120DEE720684069C0F314
:104B600080000028D3D00020D6E72DE9F04104468C
:104B70000D4617461E46DDF8188038E0701CA8B3B5
:104B8000FDF780FFA0EB0800B04200D876BBC5F36C
:104B9000074001280AD120684069A9B20840A9B29B
:104BA000884201D101200BE0002009E020688069E3
:104BB000A9B20840A9B2884201D1012000E000203A
:104BC000B84214D100202063202084F83D0000204A
:104BD00084F83E00206C40F02000206400BF0020DC
:104BE00084F83C0000BF0120BDE8F081FFE7C5F379
:104BF000074001280AD120684069A9B20840A9B23B
:104C0000884201D101200BE0002009E02068806982
:104C1000A9B20840A9B2884201D1012000E00020D9
:104C2000B842ABD00020DFE72DE9F04104460D4645
:104C300016461F4658E020684069C0F38020E8B15E
:104C40002068006840F40070216808606FF480609C
:104C50002168486100202063202084F83D00002066
:104C600084F83E00206C40F00400206400BF002067
:104C700084F83C0000BF0120BDE8F081701C90B3B7
:104C8000FDF700FFC01BB04200D866BBC5F307406C
:104C900001280AD120684069A9B20840A9B2884217
:104CA00001D101200BE0002009E020688069A9B251
:104CB0000840A9B2884201D1012000E0002090B94B
:104CC00000202063202084F83D00002084F83E006E
:104CD000206C40F02000206400BF002084F83C00DD
:104CE00000BF0120C8E7FFE7C5F3074001280AD14C
:104CF00020684069A9B20840A9B2884201D10120C8
:104D00000BE0002009E020688069A9B20840A9B240
:104D1000884201D1012000E0002000288BD0002033
:104D2000AAE770B504460D46164637E0206840698C
:104D3000C0F30010A0B16FF010002168486100209E
:104D40002063202084F83D00002084F83E00206C81
:104D5000206400BF002084F83C0000BF012070BD2B
:104D6000FDF790FE801BA84200D8BDB920684069BD
:104D7000C0F3801090B900202063202084F83D000B
:104D8000002084F83E00206C40F02000206400BF2A
:104D9000002084F83C0000BF0120E0E72068406963
:104DA000C0F380100028C1D00020D8E770B50446B9
:104DB0000D46164625E02046FFF764FD08B10120A8
:104DC00070BD681CE8B1FDF75DFE801BA84200D8ED
:104DD000BDB920684069C0F3C01090B900202063BD
:104DE000202084F83D00002084F83E00206C40F034
:104DF0002000206400BF002084F83C0000BF012098
:104E0000DEE720684069C0F3C0100028D3D000203E
:104E1000D6E7000010B501F05DFA4FF48062094951
:104E20000948FFF766F909A000F01AF84FF4FA6094
:104E3000FDF70CFD08A000F013F8FCF7A3FFFDF749
:104E400017F810BDEC0500203005002041542B431D
:104E500046554E3D310D0A0041540D0A0000000038
:104E600070B504464FF400711A48FBF7E3F90020CF
:104E700019490880194908802046FBF70EFA86B2C6
:104E80004FF4FA73324621461548FFF799FC4FF468
:104E90007A7514E01148008800280DDD11A1124830
:104EA000FBF7D3F920B911A10F48FBF7CEF900B1F8
:104EB00070BD0020094908800120FDF7C7FC281EAD
:104EC000A5F101018DB2E5D121460AA002F0F0FD65
:104ED00000BFEDE76C0600205200002050000020CB
:104EE000300500204F4B0000EC0500204552524F8A
:104EF000520000004154C3FCC1EEB3ACCAB13A2029
:104F000025730A0010B50248FDF7C2FD10BD000070
:104F10002C0300201FB504464FF4FA60012103AAB8
:104F20000B46CDE9002102902246A1210348FDF75E
:104F300097FE9DF80C0004B010BD00002C0300206B
:104F4000FEB504460D4616464FF4FA60012322468C
:104F5000A121CDE9005602900148FDF781FEFEBD7A
:104F60002C03002013B584B004464FF4FA600121ED
:104F700005AA0B46CDE9002102902246A021044853
:104F8000FDF7F2FF0520FDF761FC06B010BD000043
:104F90002C030020FEB504460D4616464FF4FA6079
:104FA00001232246A021CDE9005602900348FDF7D7
:104FB000DBFF0520FDF74AFCFEBD00002C030020AE
:104FC00000B5A1B021A0FFF74BFF4FF49670FDF79D
:104FD0003DFC22A0FFF744FF4FF49670FDF736FC2E
:104FE00022A0FFF73DFF6420FDF730FC27A0FFF76C
:104FF00037FF6420FDF72AFC2CA32EA231A101A8C3
:1050000002F066FD01A8FFF72BFF4FF4FA60FDF7F1
:105010001DFC32A034A336A23AA1009001A802F0F0
:1050200057FD01A8FFF71CFF4FF47A70FDF70EFC47
:105030003CA244A101A802F04BFD01A8FFF710FF1C
:105040004FF47A70FDF702FC21B000BD41542B51A2
:105050004D54444953433D300D0A000041542B51F7
:105060004D54434C4F53453D300D0A0041542B5194
:105070004D544346473D22726563762F6D6F6465DC
:10508000222C302C302C300D0A00000041542B51C2
:105090004D544346473D226B656570616C6976658A
:1050A000222C302C36300D0A000000003138383305
:1050B000000000003130312E34362E35322E363796
:1050C0000000000041542B514D544F50454E3D308F
:1050D0002C222573222C25730D0A00006C64686253
:1050E00030383133000000006C646862000000005A
:1050F0004C444D435532303235303132304130300E
:105100003031000041542B514D54434F4E4E3D30F1
:105110002C222573222C222573222C222573220D6A
:105120000A0000002F7365727665722F636F6F2F10
:105130004C444D43553230323530313230413030CD
:105140003031000041542B514D545355423D302CC9
:10515000312C222573222C310D0A000070B5C2B00B
:10516000F7480088002875DDF649F7A002F0A0FC9A
:10517000FBA1F448FBF769F800286CD07B21F148CB
:10518000FBF781F804467D21EE48FBF78DF80546D4
:10519000002C7DD0002DFCD0A54279D9281B461CBF
:1051A0004FF4807102A8FBF745F83246214602A869
:1051B000FBF75DF80020019001AAECA102A8FBF723
:1051C0007FF8012833D10198012804D0022810D09B
:1051D00003282AD11BE0012001F072FCE6A002F0B6
:1051E00067FC0020D64908808021D648FBF722F8CA
:1051F0001CE0022001F064FCE3A002F059FC002056
:10520000CF4908808021CF48FBF714F80EE0032037
:1052100001F056FCE0A002F04BFC0020C8490880D9
:105220008021C848FBF706F800E000BF39E301AA77
:10523000DDA102A8FBF744F8012835D1DD48FEF7CF
:105240006DFDDD48007801280AD0022804D003282B
:105250000ED109E05EE356E3D8490198086007E003
:10526000D7490198086003E0D6490198086000BF5B
:1052700000BF01F027FF0020FCF7D8F80020FCF762
:105280002DF80020FCF73CF80020CF49086000E032
:1052900038E3CE490860C7490968486201F008FA56
:1052A000C448FEF7E7FCFCE201AAC9A102A8FBF78B
:1052B00007F8012831D1BF48FEF730FDBE4800781D
:1052C000012808D0022802D003280CD107E0C349E6
:1052D0000198086007E0C2490198086003E0C149ED
:1052E0000198086000BF00BF01F0ECFE0020FCF751
:1052F0009DF80020FBF7F2FF0020FCF701F80020EA
:10530000B1490860B1490860AA490968486201F0DA
:10531000CFF9A848FEF7AEFCC3E201AAB2A102A8E9
:10532000FAF7CEFF012831D1A248FEF7F7FCA248D8
:105330000078012808D0022802D003280CD107E009
:10534000AC490198086007E0AB490198086003E0A8
:10535000AA490198086000BF00BF01F0B3FE002019
:10536000FCF764F80020FBF7B9FF0020FBF7C8FF4B
:10537000002095490860954908608E49096848628F
:1053800001F096F98B48FEF775FC8AE201AA9CA110
:1053900002A8FAF795FF01282ED187480078012846
:1053A00008D0022802D003280CD107E097490198C1
:1053B000086007E096490198086003E09549019864
:1053C000086000BF00BF01F07DFE0020FCF72EF852
:1053D0000020FBF783FF0020FBF792FF00207A49B3
:1053E00008607A49086073490968486201F060F909
:1053F0007048FEF73FFC54E201AA87A102A8FAF721
:105400005FFF012831D16B48FEF788FC6A480078BD
:10541000012808D0022802D003280CD107E08149D6
:105420000198086007E080490198086003E07F491F
:105430000198086000BF00BF01F044FE0020FBF7A8
:10544000F5FF0020FBF74AFF0020FBF759FF002083
:105450005D4908605D49086056490968486201F085
:1054600027F95448FEF706FC1BE201AA70A102A826
:10547000FAF726FF012831D14E48FEF74FFC4E487F
:105480000078012808D0022802D003280CD107E0B8
:105490006A490198086007E069490198086003E0DB
:1054A00068490198086000BF00BF01F00BFE0020B2
:1054B000FBF7BCFF0020FBF711FF0020FBF720FFEC
:1054C000002041490860414908603A49096848623A
:1054D00001F0EEF83748FEF7CDFBE2E101AA5AA150
:1054E00002A8FAF7EDFE012815D10198012808D18C
:1054F00058490870002058490860012000F00AFF50
:10550000CFE101980028AFD1524908705249086094
:1055100000F000FFC5E101AA50A102A8FAF7D0FEF1
:1055200001280CD150490198086000204A490860C0
:105530004E4801684C48006801F023F9B1E197E05A
:1055400050000020EC050020BDD3CAD5B5BDB5C4C0
:10555000D4ADCABCCAFDBEDD3A2025730A000000E6
:105560002B514D54524543563A0000007B2258318E
:1055700030223A25647D0000C7D0BBBBB5BDB3E582
:10558000B2DEC4A3CABD0A00C7D0BBBBB5BDB9E07B
:10559000B8C8C4A3CABD0A00C7D0BBBBB5BDD6B18D
:1055A000C5C5C4A3CABD0A007B22583234223A259D
:1055B000647D0000800300202C010020E800002012
:1055C000C8000020A8000020300100203401002085
:1055D0007B22583235223A25647D0000EC00002001
:1055E000CC000020AC0000207B22583534223A2524
:1055F000647D0000F0000020D0000020B0000020FA
:105600007B22583535223A25647D0000F4000020C5
:10561000D4000020B40000207B22583536223A25E1
:10562000647D000000010020D8000020B8000020A8
:105630007B22583537223A25647D00000401002082
:10564000DC000020BC0000207B22583135223A25A6
:10565000647D000054010020580100207B22583254
:1056600030223A25647D00005C01002060010020AA
:1056700001AAA9A102A8FAF723FE01280CD1A94981
:10568000019808600020A8490860A6480168A7485A
:10569000006801F076F804E101AAA5A102A8FAF7D2
:1056A0000FFE012829D10198012802D00198002875
:1056B000F1D1019808B9012000E000209F4908704D
:1056C0000198012808D1002008700120FBF7AEFEE8
:1056D0009BA002F0EDF908E0012098490870002035
:1056E000FBF7A4FE9AA002F0E3F900209C49088091
:1056F00080219C48FAF79EFDD3E001AA9AA102A856
:10570000FAF7DEFD012822D10198012802D0019884
:105710000028C0D1019808B9012000E00020954977
:1057200008700198012808D1002008700120FBF7BB
:10573000D5FD91A002F0BCF9B3E001208D490870BD
:105740000020FBF7CBFD90A002F0B2F9A9E001AA7E
:1057500091A102A8FAF7B4FD01281CD101980128F3
:1057600002D00198002896D10198012809D1002083
:10577000804908700120FBF7C3FD8AA002F098F968
:105780008FE001207B4908700020FBF7B9FD89A05C
:1057900002F08EF985E001AA8AA102A8FAF790FD2D
:1057A00001280AD10198012802D00198002878D157
:1057B0000199C8B2FBF7D4FD73E001AA84A102A845
:1057C000FAF77EFD012807D19DED010AB8EEC00A67
:1057D000824880ED000A64E001AA81A102A8FAF7DC
:1057E0006FFD012807D19DED010AB8EEC00A7F4880
:1057F00080ED000A55E001AA7DA102A8FAF760FD3C
:10580000012809D10198012801D0019808BB01990C
:10581000C8B2FBF71DFD44E001AA78A102A8FAF77F
:105820004FFD012816D1019801280FD1002076499B
:1058300008607648007808B9012000E0002073492C
:105840000870FBF7BBFD00F0C1FD2AE00020FBF76C
:1058500097FD26E001AA6EA102A8FAF731FD012802
:105860000CD16E49019808600020674908606C48B7
:1058700001686A48006800F09AFF12E001AA69A175
:1058800002A8FAF71DFD01280BD1654901980860AF
:1058900000205D490860624801686048006800F0C7
:1058A00086FF01AA62A102A8FAF70AFD01280BD11E
:1058B0000198012802D1FBF7FFFC22E0019800BB10
:1058C0000020FBF7F9FC1CE001AA5CA102A8FAF792
:1058D000F7FC012815D10198012803D1042001F01B
:1058E000EFF807E0019828B9032001F0E9F856A085
:1058F00002F0DEF800201A49088080211948FAF7E2
:1059000099FC00BF00BF0020154908808021154880
:10591000FAF790FC42B070BD7B22583231223A2512
:10592000647D000060010020580100205C0100201F
:105930007B22583132223A25647D00004800002045
:10594000CBAEB1C3C7BFD6C6BFAAC6F40A0000001B
:10595000CBAEB1C3C7BFD6C6B9D8B1D50A00000017
:1059600050000020EC0500207B22583133223A25DC
:10597000647D000049000020B7E7BBFA31C7BFD6FD
:10598000C6BFAAC6F40A0000B7E7BBFA31C7BFD644
:10599000C6B9D8B1D50A00007B22583134223A2545
:1059A000647D0000B7E7BBFA32C7BFD6C6BFAAC640
:1059B000F40A0000B7E7BBFA32C7BFD6C6B9D8B100
:1059C000D50A00007B22583138223A25647D000038
:1059D0007B22583232223A25647D0000700100207B
:1059E0007B22583233223A25647D00007401002066
:1059F0007B22583539223A25647D00007B225834B9
:105A000039223A25647D0000F401002000020020C4
:105A10007B22583531223A25647D0000F8010020B0
:105A2000FC0100207B22583532223A25647D00009B
:105A30007B22583533223A25647D00007B2258357D
:105A400038223A25647D0000CDA3D6B9C5E0BEFA60
:105A5000C4A3CABDA3ACC7D0BBBBB5BDD6B1C5C579
:105A6000C4A3CABD0A00000070B506460C46154620
:105A70004FF480710E48FAF7DDFB0EA214A10C481A
:105A800002F026F80A48FFF7EBF94FF47A732A463A
:105A900021461648FEF794FE4FF47A73012214A1B2
:105AA0001248FEF78DFE6420FCF7D0FE70BD0000AA
:105AB0006C0800202F6465762F636F6F2F4C444D68
:105AC00043553230323530313230413030303100B0
:105AD00041542B514D545055423D302C302C302CDC
:105AE000302C222573220D0A000000003005002012
:105AF0001A00000010B500F07BFD04465C480078F9
:105B0000844209D000205B4908605B49086001209D
:105B10005A49087056480470002C52D158480078F1
:105B200030B10020FBF782FC0020564908601FE0DE
:105B30005048006854490968884206D20120FBF7A2
:105B400075FC01204F49086012E04F4800684F493A
:105B50000968084447490968884206D90020FBF7CC
:105B600065FC00204749086002E0002041490860C8
:105B70004748007818B10020FBF7D4FB77E03E4897
:105B8000006844490968884203D20120FBF7CAFB38
:105B90006DE00020FBF7C6FB3E4800683E490968FF
:105BA000084435490968884261D8002032490860B4
:105BB0003A48007808B9012000E000203749087011
:105BC00055E00020FBF732FC00202E4908603048E9
:105BD000007818B10020FBF7A5FB48E027480078C3
:105BE00020B3254800682E490968884203D2012065
:105BF000FBF798FB3BE00020FBF794FB284800688C
:105C00002849096808441C49096888422FD800209F
:105C1000194908602148007808B9012000E00020F7
:105C20001E49087000201549087020E012480068DD
:105C30001D490968884203D20120FBF773FB16E077
:105C40000020FBF76FFB18480068184909680844F2
:105C50000949096888420AD80020074908600F48A6
:105C6000007808B9012000E000200C49087010BD40
:105C700045010020300100203401002039010020BE
:105C80004800002040010020E8000020EC00002037
:105C900049000020F0000020F4000020380100201E
:105CA000F8000020FC00002000010020040100207A
:105CB00010B52DED028B9FED0E0AB0EE408A6420E8
:105CC000FFF728F90446A52C05D1602000F0B8FCA8
:105CD000B0EE408A07E09FED060AB0EE408AB0EED3
:105CE000480A00F030FDB0EE480ABDEC028B10BD52
:105CF0000000000010B58820FFF70CF90446A72C1F
:105D000010D1802000F09CFCBCEEC00A094880ED58
:105D1000000A842000F094FCBCEEC00A064880ED26
:105D2000000A05E0044801680248006800F029FD07
:105D300010BD00005C0100206001002010B598201B
:105D4000FFF7E8F80446B72C10D1902000F078FC5B
:105D5000BCEEC00A094880ED000A942000F070FCF7
:105D6000BCEEC00A064880ED000A05E00448016860
:105D70000248006800F01BFD10BD0000F801002083
:105D8000FC01002010B57820FFF7C4F80446A62CCB
:105D90000CD1702000F054FC094880ED000A7420FA
:105DA00000F04EFC074880ED000A07E00548D0ED02
:105DB000000A034890ED000A00F00FFD10BD00003E
:105DC00070010020740100201FB500200090019098
:105DD0000290039015481649086000204860002191
:105DE000134881600161017680F82010C162114979
:105DF00081620021C1600121C161002180F8301061
:105E000001214161FCF732F908B1FBF7D5FE002012
:105E10000090012001900020029069460448FCF7A0
:105E20005BF808B1FBF7C8FE1FBD00000020014071
:105E30003C0200200100000F1FB5002000900190DF
:105E4000029003902048214908600020486000210A
:105E50001E488160012101610176002180F8201037
:105E6000C1621B4981620021C1600321C16101211E
:105E700080F830104161FCF7F9F808B1FBF79CFE9F
:105E800004200090012001900720029069460F48ED
:105E9000FCF722F808B1FBF78FFE092000900220E2
:105EA000019069460948FCF717F808B1FBF784FE32
:105EB0000E2000900320019069460448FCF70CF87E
:105EC00008B1FBF779FE1FBD0022014084020020CB
:105ED0000100000F08B500BF0020009012480068C4
:105EE00040F40010104908600846006800F40010F3
:105EF000009000BF00BF00BF00200090084600686F
:105F000040F4800008600846006800F480000090BB
:105F100000BF00BF002211460D20FDF7A3F90D20A0
:105F2000FDF78CF908BD00003038024000B587B09D
:105F3000142102A8FAF77EF900BF0020019055480D
:105F4000006840F01000534908600846006800F0FF
:105F50001000019000BF00BF00BF00200190084664
:105F6000006840F0040008600846006800F0040083
:105F7000019000BF00BF00BF0020019008460068EC
:105F800040F0200008600846006800F02000019002
:105F900000BF00BF00BF002001900846006840F02D
:105FA000800008600846006800F08000019000BF93
:105FB00000BF00BF002001900846006840F00100CB
:105FC00008600846006800F00100019000BF00BFB3
:105FD00000BF002001900846006840F040000860C3
:105FE0000846006800F04000019000BF00BF00BFFD
:105FF000002001900846006840F00800086008464C
:10600000006800F00800019000BF00BF00220C21D2
:106010002148FCF731FD002242F65E211F48FCF7C3
:106020002BFD0C200290012003900020049005908D
:1060300002A91948FCF71EFC0420029000200390DE
:10604000049002A91648FCF715FC202002900020BD
:1060500003900120049002A91248FCF70BFC40F6C3
:106060001E2002900120039000200490059002A9B8
:106070000A48FCF7FFFB4FF4015002900120039007
:10608000002004900220059002A90448FCF7F2FBCE
:1060900007B000BD30380240001002400018024036
:1060A000001402400008024010B50B480B4908607C
:1060B0000B484860002109488160C1604FF480416D
:1060C0000161002141618161C1610162FCF7E0FC75
:1060D00008B1FBF771FD10BD005800402C030020F3
:1060E000A086010000B587B00020039004900590C1
:1060F0000690019002904FF080401449086041F6EC
:106100001F4048600021114881601149C160002191
:1061100001618161FDF7FCFC08B1FBF74DFD4FF417
:106120008050039003A90948FDF717FE08B1FBF75B
:1061300043FD00200190029001A90448FDF78EFC68
:1061400008B1FBF739FD07B000BD00008003002057
:10615000BF27090000B587B0002003900490059088
:1061600006900190029015481549086041F61F40BD
:10617000486000211248816042F20F71C160002125
:1061800001618161FDF7C4FC08B1FBF715FD4FF417
:106190008050039003A90A48FDF7DFFD08B1FBF723
:1061A0000BFD00200190029001A90548FDF756FC67
:1061B00008B1FBF701FD07B000BD0000000400407E
:1061C000C80300201CB50020009001900E480F4924
:1061D00008604720486000210C48816040F2E731A8
:1061E000C16000218161FDF793FC08B1FBF7E4FC7D
:1061F00000200090019069460448FDF72FFC08B18B
:10620000FBF7DAFC1CBD0000001000401004002069
:106210001CB50020009001900E480F49086041F61F
:106220001F40486000210C48816042F20F71C1603C
:1062300000218161FDF76CFC08B1FBF7BDFC00207B
:106240000090019069460448FDF708FC08B1FBF78F
:10625000B3FC1CBD001400405804002010B50D48CC
:106260000D4908604FF4965048604FF480510A4839
:1062700081600021C1604FF4806101610C214161A6
:1062800000218161C161FEF7FBF808B1FBF794FCC6
:1062900010BD0000004C0040A004002010B50B48C9
:1062A0000B4908604FF4E1304860002108488160E4
:1062B000C16001610C21416100218161C161FEF772
:1062C000DFF808B1FBF778FC10BD000000100140BA
:1062D000E804002010B50B480B4908604FF4E1308A
:1062E0004860002108488160C16001610C21416162
:1062F00000218161C161FEF7C3F808B1FBF75CFCC6
:1063000010BD0000004400403005002000BFFEE743
:1063100000BFFEE710B504462CB10122402105481C
:10632000FCF7AAFB04E0002240210248FCF7A4FB92
:1063300010BD00000018024010B512480078E8B106
:106340001148006811490968884203D80120FFF705
:10635000E1FF16E00D4800680D49096808440A4944
:106360000968884203D30020FFF7D4FF09E000202A
:10637000054908600120FFF7CDFF02E00020FFF78C
:10638000C9FF10BD54010020580100205C0100200D
:106390006001002010B540210148FCF765FB10BDED
:1063A0000018024010B5FFF7A5FC01200449087051
:1063B0000020044908600120FFF7ACFF10BD000079
:1063C00054010020580100207047000010B5174804
:1063D000006817490968884206D80120FAF7D0FFFB
:1063E0000120144908701FE011480068124909682B
:1063F00008440E490968884206D30020FAF7C0FF16
:1064000000200C4908700FE00020084908600B4884
:10641000007808B9012000E0002008490870FAF768
:10642000CDFF0120FAF7ACFF10BD0000F401002001
:10643000F801002001020020FC01002000020020E1
:1064400010B5FFF77BFC0020044908600449087080
:10645000FAF7B4FF0120FAF793FF10BDF401002012
:106460000002002070B52DED108B04469FED400A10
:10647000B0EE40FA208808EE100AB8EE480ADFEDC8
:106480003D0A20EE200ADFED3A0A20EE200A3A48C3
:1064900080ED000A90ED000ADFED380A20EE200AB8
:1064A000D0ED000A9FED361A71EE600A80EE201AD8
:1064B000F0EE418A9FED310AC8EE800A10EE905A44
:1064C0002846FAF76DF941EC1E0BB0EE4E0AF0EEDD
:1064D0006E0A01F02DFBB0EE40DAF0EE60DA9FEDCF
:1064E000290B53EC102B51EC1D0BFAF7C4F841ECBF
:1064F0001C0B9FED260B53EC102BF9F7A3FF41EC7F
:106500001B0B53EC1B2B9FED230B51EC100BFAF7DD
:10651000B2F841EC1A0B9FED210B53EC102BFAF75C
:1065200032F841EC190BFAF767F91E490860084682
:1065300090ED000A1C48D0ED000AB4EEE00AF1EE3E
:1065400010FA03D20120FAF70BFF0DE0154890ED89
:10655000000A1648D0ED000AB4EEE00AF1EE10FA97
:1065600002DD0020FAF7FCFEBDEC108B70BD0000D0
:106570009A99193F3333533A7801002000401C4662
:10658000333353400000000000DCAE40000000E068
:10659000E1796B3F000000000000F03F0000006068
:1065A000661271407C0100207001002074010020FF
:1065B00010B510210148FCF757FA10BD0018024031
:1065C00010B504210148FCF74FFA10BD0018024035
:1065D00010B508210148FCF747FA10BD0018024029
:1065E00010B520210148FCF73FFA10BD0008024019
:1065F00010B5FFF7F5FF04460E480078844205D039
:1066000000200D4908700B48047010E00A4800781B
:106610000A280CDA08480078401C07490870084628
:1066200000780A2803DB054804700020087003483E
:10663000007810BD3B0100203A0100203C01002001
:106640001CB50446042201A92046FEF779FC0198F6
:1066500000909DED000A1CBD10B54FF4007102487A
:10666000FCF702FA10BD00000018024010B504212A
:106670000148FCF7F9F910BD0014024010B50421DF
:106680000648FCF7F1F920B908210448FCF7ECF9B9
:1066900008B1012010BD0020FCE7000000100240FE
:1066A00010B502210148FCF7DFF910BD00180240C7
:1066B00010B51B48FDF732FB00F0D8F9002019494E
:1066C00008601949086019490860194908600120E3
:1066D00018490870002018490860184908704FF4DC
:1066E0007A70FCF7B3F816480078012804D0022825
:1066F00005D0032809D105E000F026FA05E000F0F6
:1067000043FA02E000F006FA00BF00BF002005498E
:106710000860054908600248FDF7ACFA10BD0000AA
:1067200080030020300100203401002024010020DB
:1067300028010020390100204001002038010020FC
:106740002C010020704710B52DED028BB0EE408A71
:10675000B0EE480A602000F007F8A5216420FEF79B
:1067600001FCBDEC028B10BD11B52DED020B81B00B
:10677000044601980090042269462046FEF70AFC70
:106780001FBD70B504460D4600EE104AB8EE400A33
:106790008020FFF7E9FF00EE105AB8EE400A84208F
:1067A000FFF7E2FFA7218820FEF7DCFB70BD70B584
:1067B00004460D4600EE104AB8EE400A9020FFF75E
:1067C000D3FF00EE105AB8EE400A9420FFF7CCFF3A
:1067D000B7219820FEF7C6FB70BD10B52DED028BDA
:1067E000F0EE408AB0EE608AB0EE680A7020FFF7E3
:1067F000BBFFB0EE480A7420FFF7B6FFA621782051
:10680000FEF7B0FBBDEC028B10BD000010B5FFF72A
:10681000EFFE044680480078844207D000207F497C
:10682000086001207E4908707B48047014BB7B48D7
:1068300000687C490968884203D20120FAF772FD9A
:1068400063E0784800687849096808447349096832
:10685000884203D90020FAF765FD56E000206F4911
:1068600008607248007808B9012000E000206F49F4
:1068700008704AE06A48007828B3684800686C49A4
:106880000968884203D20120FAF74CFD3DE06848D0
:10689000006868490968084460490968884203D962
:1068A0000020FAF73FFD30E000205C4908605F48B7
:1068B000007808B9012000E000205C490870002041
:1068C0005749087021E0554800685B4909688842CB
:1068D00003D20120FAF726FD17E057480068574910
:1068E000096808444D490968884203D90020FAF72D
:1068F00019FD0AE00020494908604C48007808B9B1
:10690000012000E00020494908704D48007830B16E
:10691000012819D0022847D003287BD174E0002039
:10692000FAF784FD00204749086047480068474956
:106930000968884207D9012041490870002042496E
:1069400008604349086065E03F48006841490968BC
:10695000884220D23E4800683F490968884206D2F2
:106960000120FAF763FD0120364908601BE03A4830
:1069700000683A490968084435490968884206D9D7
:106980000020FAF753FD00202E4908600BE000209C
:106990002F49086007E002202949087000202A4991
:1069A00008602B49086035E0274800682C490968D1
:1069B000884220D22648006827490968884206D2C2
:1069C0000120FAF733FD01201E4908601BE0224830
:1069D00000682449096808441D490968884206D9A5
:1069E0000020FAF723FD0020164908600BE0002084
:1069F0001749086007E003201149087000F08AF881
:106A000003201949087005E000F084F803201649B6
:106A1000087000BF00BF10BD4701002034010020F6
:106A200039010020B0000020B4000020380100200F
:106A3000C0000020C4000020B8000020BC000020DE
:106A40002001002040010020240100200801002036
:106A5000280100200C01002010010020140100205A
:106A6000180100201C0100202C01002010B500207E
:106A7000FAF7DCFC0020FAF731FC0020FAF740FCC2
:106A80000020094908600949086009490860094966
:106A900008600120084908700020084908604FF488
:106AA0007A70FBF7D3FE10BD3001002034010020C6
:106AB000240100202801002039010020400100208D
:106AC00010B50446FFF7D2FF012C06D0022C0AD0E5
:106AD000032C0ED0042C18D111E000F035F8012061
:106AE0000B49087012E000F04FF8022008490870C6
:106AF0000CE000F00FF803200549087006E000F0F4
:106B000063F804200249087000E000BF00BF10BD18
:106B10002C01002010B500200849086008490860D1
:106B2000FFF766FD074908700020FAF77FFC002098
:106B3000FAF7D4FB0020FAF7E3FB10BD3001002088
:106B4000340100204401002010B500200A490860EB
:106B50000A49086001200A490870FFF749FD094900
:106B600008700020FAF762FC0020FAF7B7FB00205B
:106B7000FAF7C6FB10BD00003001002034010020F0
:106B8000390100204601002010B500200A490860A4
:106B90000A49086001200A490870FFF729FD0949E0
:106BA00008700020FAF742FC0020FAF797FB00205B
:106BB000FAF7A6FB10BD00003001002034010020D0
:106BC000390100204501002010B500200D49086062
:106BD0000D4908700D4908600D49086001200D49F4
:106BE0000870FFF705FD0C4908700020FAF71EFC3D
:106BF0000020FAF773FB0020FAF782FB0420074914
:106C0000087010BD34010020200100202401002064
:106C10002801002039010020470100202C0100201C
:106C200010B5FCF797FA10BD00B593B0302107A856
:106C3000F9F700FB142102A8F9F7FCFA00BF0020C5
:106C400001902348006840F08050214908600846C0
:106C5000006800F08050019000BF00BF00BF00201E
:106C600001901C48006840F480401A4908600846BA
:106C7000006800F48040019000BF00BF0120079031
:106C80000004089002200D9041050E9108210F91FB
:106C900090211091022111910421129107A8FCF773
:106CA00073FC08B1FAF788FF0F20029002200390CE
:106CB000002004904FF4805005900020069002219F
:106CC00002A8FCF721FB08B1FAF776FF13B000BD6C
:106CD00040380240007000400348006840F47000F3
:106CE000014908607047000088ED00E010B50248D7
:106CF000FDF7BAF810BD00008003002010B502486F
:106D0000FDF7B2F810BD0000C803002010B502481E
:106D1000FDF7AAF810BD00001004002010B50248CD
:106D2000FDF7A2F810BD00005804002010B502685D
:106D30002D4B98420ED0B0F1804F0BD02B4B984288
:106D400008D02B4B984205D02A4B984202D02A4BB0
:106D5000984203D122F070024B681A43224B9842AA
:106D600020D0B0F1804F1DD0204B98421AD0204B3C
:106D7000984217D01F4B984214D01F4B984211D005
:106D80001E4B98420ED01E4B98420BD01D4B984282
:106D900008D01D4B984205D01C4B984202D01C4B8A
:106DA000984203D122F44072CB681A4322F0800348
:106DB0004C6943EA040202608B68C3620B68836219
:106DC000094B984202D00C4B984201D10B690363E6
:106DD00001234361036903F001031BB1036923F03D
:106DE0000103036110BD00000000014000040040E9
:106DF00000080040000C0040000401400040014039
:106E0000004401400048014000180040001C0040C0
:106E10000020004030B50C46816821F47F4142EAF1
:106E2000032525432943816030BD0A46816821F04E
:106E3000700142F0070319438160704730B50B467B
:106E40001446026A056A25F001050562816921F090
:106E5000F00141EA041122F00A021A438161026240
:106E600030BD30B50B461446026A056A25F01005A0
:106E70000562816921F4704141EA043122F0A002E7
:106E800042EA03128161026230BD000010B50422A3
:106E90006E490020FEF754F804226D491046FEF7B3
:106EA0004FF804226B490820FEF74AF804226A4989
:106EB0000C20FEF745F8042268491020FEF740F840
:106EC000042267491420FEF73BF804226549182084
:106ED000FEF736F8042264491C20FEF731F804223C
:106EE00062492020FEF72CF8042261492420FEF795
:106EF00027F804225F492820FEF722F804225E4981
:106F00002C20FEF71DF804225C493020FEF718F80B
:106F100004225B493420FEF713F804225949382033
:106F2000FEF70EF8042258493C20FEF709F8042227
:106F300056494020FEF704F8042255494420FDF745
:106F4000FFFF042253494820FDF7FAFF042252496B
:106F50004C20FDF7F5FF042250495020FDF7F0FFCB
:106F600004224F495420FDF7EBFF04224D495820DD
:106F7000FDF7E6FF04224C495C20FDF7E1FF3348B2
:106F80000068401C18B13148006800285CD101201D
:106F90002E49086096202E49086028202D49086057
:106FA00002202D4908600A202C49086014202C4931
:106FB000086028202B49086002202B490860012026
:106FC0002A49086096202A49086028202949086033
:106FD000022029490860052028490860192028490D
:106FE00008602820274908600220274908600120FE
:106FF0002649086078202649086014202549086041
:107000000520254908600A202649086026490860AD
:107010000520224908602820214908604FF4B46007
:107020002249086040002249086001202149086087
:107030004FF4B47020490860012020490860F02016
:107040001F49086000F03EF810BD0000A8000020B5
:10705000AC000020B0000020B4000020B8000020E8
:10706000BC000020C0000020C4000020C800002098
:10707000CC000020D0000020D4000020D800002048
:10708000DC000020E0000020E4000020E8000020F8
:10709000EC000020F0000020F4000020000100209F
:1070A00004010020F8000020FC000020080100205E
:1070B0000C01002010010020140100201801002004
:1070C0001C01002010B504223B490020FDF762FF9F
:1070D00004223A491046FDF75DFF04223849082092
:1070E000FDF758FF042237490C20FDF753FF042217
:1070F00035491020FDF74EFF042234491420FDF7D6
:1071000049FF042232491820FDF744FF0422314987
:107110001C20FDF73FFF04222F492020FDF73AFFF6
:1071200004222E492420FDF735FF04222C49282073
:10713000FDF730FF04222B492C20FDF72BFF042202
:1071400029493020FDF726FF042228493420FDF785
:1071500021FF042226493820FDF71CFF042225497F
:107160003C20FDF717FF042223494020FDF712FFC2
:10717000042222494420FDF70DFF04222049482023
:10718000FDF708FF04221F494C20FDF703FF0422EE
:107190001D495020FDF7FEFE04221C495420FDF736
:1071A000F9FE04221A495820FDF7F4FE0422194979
:1071B0005C20FDF7EFFE10BDA8000020AC00002011
:1071C000B0000020B4000020B8000020BC00002067
:1071D000C0000020C4000020C8000020CC00002017
:1071E000D0000020D4000020D8000020DC000020C7
:1071F000E0000020E4000020E8000020EC00002077
:10720000F0000020F4000020000100200401002014
:10721000F8000020FC00002010B50248FCF7BCFF7D
:1072200010BD0000A004002070B50546AC6B002026
:10723000E085E0842046FCF7ADFF70BD00BF00BFD5
:1072400002680C3252E8002F22F4907102680C326E
:1072500042E80013002BF3D100BF00BF00BF02685B
:10726000143252E8002F22F001010268143242E881
:107270000013002BF3D100BF016B01290ED100BF19
:1072800000BF02680C3252E8002F22F010010268A1
:107290000C3242E80013002BF3D100BF202180F80C
:1072A000421000210163704710B504462068C06891
:1072B00020F040002168C860202084F8410020466A
:1072C000FDF7DDFA002010BDF8B5044694F8420041
:1072D000222875D1A068B0F5805F0CD1206950B923
:1072E0000025A66A20684068C0F308003080A06AC4
:1072F000801CA06215E0A56A0026A068B0F5805F3A
:1073000003D0A06828B9206918B92068406828709F
:1073100004E02068406800F07F002870A06A401CEC
:10732000A062E08D401E80B2E085002846D1206832
:10733000C06820F020002168C8602068C06820F480
:1073400080702168C8602068406920F001002168D1
:107350004861202084F8420000206063206B0128EF
:1073600026D10020206300BF00BF21680C3151E806
:10737000001F21F0100021680C3141E80002002AB2
:10738000F3D100BF2068006800F0100010280AD177
:1073900000BF0020009020680068009020684068CE
:1073A000009000BF00BFA18D2046FCF7DBFE02E08D
:1073B0002046FDF7C1F90020F8BD01E00020FBE701
:1073C0000220F9E72DE9F84F04462068006920F40F
:1073D0004050E1680843216808612169A0680843BA
:1073E00061690843E169084300902068C06849F278
:1073F0000C618843009908432168C860206840698F
:1074000020F44070A16908432168486176492068EA
:10741000884203D075492068884203D1FCF74CF8B4
:10742000814602E0FCF738F88146E069B0F5004F8C
:107430006CD102206168A0FB015003461920A9FB12
:10744000007001462A463846F8F7BCFE6421B0FBBE
:10745000F1F04FEA001A02206168A0FB01510B46CF
:107460001920A9FB00712A463846F8F7ABFE83467F
:1074700002206168A0FB015003461920A9FB00719E
:107480002A463846F8F79EFE6421B0FBF1F000EB87
:10749000C00101EB0010ABEB8000322101EBC0001A
:1074A0006421B0FBF1F000F0F8000AEB400A022082
:1074B0006168A0FB015003461920A9FB007001463A
:1074C0002A463846F8F77EFE834602206168A0FB14
:1074D000015003461920A9FB00712A463846F8F7E7
:1074E00071FE6421B0FBF1F000EBC00101EB001074
:1074F000ABEB8000322101EBC0006421B0FBF1F066
:1075000000F007005044216888606AE00420616848
:10751000A0FB015003461920A9FB007001462A4632
:107520003846F8F74FFE824604206168A0FB015000
:1075300003461920A9FB007001462A463846F8F791
:1075400041FE6421B0FBF1F000EBC00101EB001043
:10755000AAEB8000322101EB00106421B0FBF1F0B6
:1075600000F0F00A04206168A0FB017003461920B6
:10757000A9FB00513A462846F8F724FE6421B0FBE7
:10758000F1F00AEB001A04206168A0FB01510B46E0
:107590001920A9FB00712A463846F8F713FE8346E6
:1075A00004206168A0FB015003461920A9FB00706C
:1075B00001462A463846F8F705FE6421B0FBF1F093
:1075C00000EBC00101EB0010ABEB8000322101EBBE
:1075D00000106421B0FBF1F000F00F00504421686E
:1075E0008860BDE8F88F00000010014000140140E1
:1075F00010B5034699629A85DA85002058642220E6
:1076000083F84200186928B11868C06840F4807097
:107610001C68E0601868406940F001001C68606107
:107620001868C06840F020001C68E060002010BDB1
:10763000014691F84100212828D18868B0F5805F83
:107640000BD1086948B90A6A1088C0F308000B68B2
:107650005860086A801C086205E00B6A581C0862C2
:1076600018780B685860C88C401E80B2C88458B91E
:107670000868C06820F080000B68D8600868C0689F
:1076800040F040000B68D860002070470220FCE703
:107690002DE9F84304460D4617469846089E31E00A
:1076A000701C70B3FBF7EEF9A0EB0800B04200D8F5
:1076B00016B90320BDE8F8832068C06800F0040014
:1076C000F8B1802D1ED0402D1CD020680068C0F37A
:1076D000C000B0B100BF002000902068006800909A
:1076E00020684068009000BF00BF2046FFF7A6FD5D
:1076F0000820606400BF002084F8400000BF012023
:10770000D8E7FFE7206800682840A84201D101209F
:1077100000E00020B842C3D00020CBE710B50248FB
:10772000FCF73AFD10BD00003005002010B51648EA
:10773000007816490870FEF7B3FF14494870FEF749
:107740003FFF12498870FEF743FF1049C870FEF7EB
:1077500021FE0E490871FEF743FF0C494871FEF700
:107760007BFF0A49C871FEF781FF08490872FEF7DE
:1077700085FF06494872FEF71BFF044988720448DA
:107780000078C87210BD00006C0000206C09002059
:10779000810000202DE9F04F2DED068BE5B0FFF7BD
:1077A000C5FFF9F717FDFAF721FB05467848FEF704
:1077B00059FEFAF75DFB00260027B046B146B246F7
:1077C000B34674480078012817D0022804D0032853
:1077D00024D0042864D132E06F4806686F480768F7
:1077E0006F48D0F800806F48D0F800906E48D0F80D
:1077F00000A06E48D0F800B052E06D4806686D48B1
:1078000007686D48D0F800806C48D0F800906C484C
:10781000D0F800A06B48D0F800B041E06A48066894
:107820006A4807686A48D0F800806A48D0F8009033
:107830006948D0F800A06948D0F800B030E064484A
:10784000D0F800806348D0F800906348D0F800A0DA
:107850006248D0F800B06248007820B1012809D011
:10786000022817D10EE05FA000F022F9002665483B
:10787000076813E064A000F01BF96B4806686B48CA
:1078800007680BE06AA000F013F9674806687048C3
:10789000076803E06FA000F00BF900BF00BF00BF56
:1078A00000BF73480068F8F77BFF41EC180B714884
:1078B0000068F8F775FF41EC190B6F480068F8F79E
:1078C0006FFF41EC1A0B6D4824906D4890ED000B52
:1078D0008DED220B6B48C07A2E490978042901D11D
:1078E000012100E00021CDE91DABCDE91F10654865
:1078F000807A65490968CDE91B89CDE9191063488B
:1079000001686048407A624A1278CDE91552CDE9A3
:1079100017015C48007A5B4949795E4A92785D4B71
:107920005B78CDE91132CDE913105A480078CDE9E2
:107930000E6710908DED0C8B8DED0A9B8DED08ABD5
:1079400055480168554802684E48C079544B1B7829
:10795000CDE90330CDE905214A48C1788078494A0C
:107960005278CDE9002002910A4803784D4890F9F9
:1079700000204D4925A800F0ABF884B2224625A985
:107980000020FEF771F865B0BDEC068BBDE8F08F06
:10799000100000202C010020E8000020EC00002056
:1079A000F0000020F400002000010020040100206D
:1079B000C8000020CC000020D0000020D40000200F
:1079C000D8000020DC000020A8000020AC0000202F
:1079D000B0000020B4000020B8000020BC0000204F
:1079E00020010020CCD8CAE2C4A3CABDB3F5CABCEA
:1079F000BDD7B6CE202D203234D0A1CAB1CDA3D66A
:107A0000B90A000008010020CCD8CAE2C4A3CABD4C
:107A1000B5DAD2BBBDD7B6CE202D2036D0A1CAB1A3
:107A2000D1ADBBB70A0000001001002014010020F6
:107A3000CCD8CAE2C4A3CABDB5DAB6FEBDD7B6CEAD
:107A4000202D2034D0A1CAB1D1ADBBB70A000000AF
:107A50001C010020B4EDCEF3A3BACEDED0A7B5C48E
:107A6000CCD8CAE2C4A3CABDBDD7B6CE0A000000B6
:107A700074010020700100207C010020D805002046
:107A8000C80100206C090020FC010020F801002042
:107A90000102002082000020600100205C01002023
:107AA0005401002055000020708B000800BFFEE745
:107AB0000FB4054B10B503A9044A029800F0A4FBCB
:107AC00010BC5DF814FB0000198900083402002086
:107AD0000FB4084B10B504A902AA039800F094FB58
:107AE000044602A9002000F012FF204610BC5DF8F9
:107AF00014FB00000F89000802480068C0F3022050
:107B0000704700000CED00E010B5002804DB0A0708
:107B1000130E054A135406E00A07140E034A00F038
:107B20000F031B1FD45410BD00E400E018ED00E06B
:107B300070B5D94B00242DED020B2DED108BDDE936
:107B40001010984205DA20F000429A4201D809D17B
:107B500041B19DED100BBDEC108B02B0BDE8704043
:107B600000F05EBAB0F5801F26DA11430BD0002872
:107B700013DA012000F080FABDEC108B02B0BDE8F2
:107B8000704000F059BA022000F076FA00F030FAA6
:107B900051EC100B81F000419EE06FF035049FED39
:107BA000C00B53EC102B9DED100B51EC100BF8F7A4
:107BB000F0FCCDE91001084604EB2051C0F313049A
:107BC000B948A1F2FF31204400F4801080F07F62B8
:107BD00082F04052224301EB20559FEDB50B1192EC
:107BE00053EC102B9DED100B51EC100BF8F7CBFC68
:107BF00041EC180BA01CC0F313009FEDAFDB9FED11
:107C0000B0EBB14E7E4403286CD296ED000B51ECE4
:107C1000180B53EC102BF8F753FF1DD1002D01BFAB
:107C200096ED000BBDEC108B02B070BD2846F8F746
:107C30001DFF41EC180B53EC1D2BF8F7AAFC41EC8F
:107C4000190B53EC1E2B51EC180BF8F7A2FC53EC5C
:107C5000192BF8F7F7FB3FE09FED9D0B51EC180B4C
:107C600053EC102BF8F795FC9FED9B1B53EC112B5D
:107C7000F8F78CFC41EC190B53EC182B51EC180B5A
:107C8000F8F787FC53EC192BF8F783FC41EC190B40
:107C9000002D04BF53EC192B51EC180B1AD02846B9
:107CA000F8F7E4FE41EC1A0B53EC1D2BF8F771FCCE
:107CB00053EC192BF8F76AFC53EC182BF8F763FC1C
:107CC00041EC180B53EC1E2B51EC1A0BF8F761FC2E
:107CD00053EC182BF8F757FCBDEC108B02B041ECBD
:107CE000100B70BD9FED7E0B51EC180B53EC102B5D
:107CF000F8F7A8FB41EC100B51EC180B53EC102BD0
:107D0000F8F7B9FC41EC190B2846F8F7AFFE41EC47
:107D10001B0B53EC192B51EC190BF8F73AFC41EC07
:107D20001A0B714853EC1A2B261851EC1A0BF8F762
:107D300030FC41EC1F0B6D48C4F1510404F5D7240D
:107D4000B0EE4F0AF0EE6F0A0321784400F0D2F84B
:107D500053EC1F2B51EC100BF8F71BFC41EC1C0BE8
:107D60006348B0EE4F0AF0EE6F0A0421784400F049
:107D7000C1F853EC1A2B51EC100BF8F70AFC344302
:107D800053EC1C2BF8F75EFB41EC1C0B002C4CDD7C
:107D90009FED510B51EC180B53EC102BF8F7F9FB3E
:107DA00053EC182BF8F7F5FB41EC1A0B55B353ECD9
:107DB0001D2B51EC1B0BF8F7ECFB41EC1D0B53ECAE
:107DC0001C2B51EC1A0BF8F73DFB53EC192BF8F771
:107DD000E0FB53EC1D2BF8F735FB53EC1A2BF8F7AF
:107DE000D5FB53EC182BF8F7CEFB41EC180B53ECFA
:107DF0001E2B51EC1B0BF8F7CCFB53EC182BF8F7B0
:107E0000C2FB69E753EC1C2B51EC1A0BF8F71AFB79
:107E100053EC192BF8F7BDFB53EC1A2BF8F7B6FB14
:107E200053EC182BF8F7B2FB56E735B353EC1D2B88
:107E300051EC1B0BF8F7ADFB41EC1A0B53EC1C2B70
:107E400051EC180BF8F79FFB53EC192BF8F7A1FB3B
:107E500053EC1A2BF8F797FB53EC182BF8F793FB1E
:107E600041EC180B53EC1E2B51EC1B0BF8F791FB5C
:107E700053EC182BF8F787FB2EE753EC1C2B51EC37
:107E8000180BF8F780FB53EC192BF8F782FB53EC37
:107E9000182BF8F77BFB1FE70000F07F00000000C5
:107EA0000000000000005043645F09000000000073
:107EB000000000000000F03F763C7935EF39EA3DE4
:107EC0000000E0FE422EE63F200F00000000000010
:107ED000555555555555D53F000000000000E03F71
:107EE000000000000000004086EBF9FFA20D00003A
:107EF000980D000070B504462DED028B4D1E00EB71
:107F0000C500B0EE408AF0EE608A90ED000B35F0CF
:107F1000060017D053EC182B51EC100BF8F739FB77
:107F200041EC100B6D1E04EBC50090ED001B51ECF5
:107F3000100B53EC112BF8F785FA41EC100B35F0D0
:107F40000600E7D1022D36D0042D1CD0062D1CBF13
:107F5000BDEC028B70BD53EC182B51EC100BF8F7F5
:107F600018FB94ED0A1B53EC112BF8F76BFA53EC4A
:107F7000182BF8F70EFB94ED081B53EC112BF8F7B8
:107F800061FA41EC100B53EC182B51EC100BF8F785
:107F900000FB94ED061B53EC112BF8F753FA53EC4E
:107FA000182BF8F7F6FA94ED040B53EC102BF8F7B6
:107FB00049FA41EC100B53EC182B51EC100BF8F76D
:107FC000E8FA94ED021B53EC112BF8F73BFA53EC53
:107FD000182BF8F7DEFA94ED001B53EC112BF8F791
:107FE00031FABDEC028B41EC100B70BD00000000BB
:107FF0009FED070B10B553EC102B9FED070B51ECC9
:10800000100BF8F738FB41EC100B10BD000000001E
:108010000000000000000000000000000000F03F31
:1080200010B553EC102B51EC100BF8F70BFA41EC98
:10803000100B10BD000000009FED050B10B553ECB8
:10804000102B51EC100BF8F716FB41EC100B10BD88
:10805000000000000000000002E008C8121F08C174
:10806000002AFAD170477047002001E001C1121FB9
:10807000002AFBD1704700000149086070470000EA
:10808000380200202DE9FF5F82B00021DDE90430D5
:10809000020DDDF840B0034318D044F61050A2F2B0
:1080A000FF3242431514119801281FD0A5EB0B0095
:1080B000401C5FEA000A4FF000064E4FDFF838918F
:1080C000B046504615D5CAF1000413E011980124BA
:1080D0004AA3012801D16FEA0B010298119AC0E965
:1080E0000031C0E9024206B0BDE8F09FCBF10000CC
:1080F000DFE704460021404A491842EB0450CDE92D
:10810000001012E0E00707D032463B4640464946A1
:10811000F8F73FFA8046894632463B4610461946F4
:10812000F8F737FA06460F466410002CEAD1DDE96D
:108130000401DDE90023BAF1000F06DAF8F729FAA5
:1081400042464B46F8F725FA05E0F8F794FA42461E
:108150004B46F8F790FA04460E460022284BF8F7F3
:1081600033FB03D84FF0FF30014607E00022254BD8
:1081700020463146F8F766F9F8F789FC102409E043
:10818000002C0ADB0A220023F8F71CF8039B30328C
:108190001A55641E50EA0102F2D1641C039AC4F11C
:1081A00011031444119A012A03D0012208430DD16E
:1081B0000AE0084304D000204FF0110B119072E741
:1081C000A3EB0B056D1E0DE05B4504DD4FF00002D7
:1081D00005F1010504E003DA4FF00002A5F1010505
:1081E000002AECD002981199C0E90231C0E900459B
:1081F00079E70000000014400000F03F300000006C
:108200000000F0430000E03F2DE9FF4F95B09A4693
:10821000884606460025EEE1252877D1002427462A
:10822000F94A0121039400E0044316F8013F203B82
:1082300001FA03F01042F7D130782A2811D06FF0FC
:108240002F033078A0F13002092A16D8039A44F09F
:10825000020402EB820203EB42021044761C0390FC
:10826000EFE758F8042B0392002A03DA504244F453
:108270000054039044F00204761C30782E2816D166
:1082800016F8010F44F004042A280DD06FF02F02D5
:108290003078A0F13003092B09D807EB870302EBF4
:1082A0004303C718761CF3E758F8047B761C307834
:1082B0006C280FD006DC4C2817D068280DD06A280F
:1082C00014D104E0742810D07A280FD10DE044F4C2
:1082D00000140AE044F4801401E044F4401472787D
:1082E000824202D104F58014761C761C3078662810
:1082F0000BD013DC582877D009DC002875D045282E
:10830000F6D04628F4D047281AD193E118E0632824
:1083100035D0642879D0652812D18BE1702873D0CC
:1083200008DC6728F1D069286FD06E280DD06F283F
:1083300006D1ACE073282CD0752874D0782853D09F
:108340005246179990476D1C54E1C4F3025002281D
:1083500009D003280DD0D8F8001004280DD00D60E6
:1083600008F1040846E1D8F80010EA17C1E9005204
:10837000F6E7D8F800100D80F2E70D70F0E718F876
:10838000041B8DF8001000208DF80100EB46012041
:1083900003E058F804BB4FF0FF3061074FF00001D5
:1083A00002D40DE009F101018946B9420FDA814595
:1083B000F8DB1BF809100029F4D108E009F10101EC
:1083C00089468142FADB1BF809100029F6D103988F
:1083D0005346A0EB090721463846179A00F080FA69
:1083E000284400EB090507E044E008E10DE01BF834
:1083F000010B524617999047B9F10109F7D253463C
:1084000021463846179AF2E039E00A21C4F30252B5
:108410004FF0000B0091022A06D058F8040BC11748
:10842000032A09D00AE023E008F1070020F0070240
:10843000F2E80201904605E000B2C117042A01D11A
:1084400040B2C117002906DA0A460021404261EB1A
:1084500002012D2202E0220504D52B228DF80420F2
:10846000012203E0E20701D02022F7E7914657E01E
:108470000A2100E010214FF0000B00910BE01021C9
:108480004FF0000B44F004040827009103E008209B
:108490004FF0000B0090C4F30252022A05D058F8A6
:1084A000040B0021032A08D008E008F1070020F09F
:1084B0000702F2E80201904603E080B2042A00D1EC
:1084C000C0B24FF0000922072AD53278702A07D0AF
:1084D000DDF800C08CF0100C5CEA0B0C05D00EE04F
:1084E00040228DF80420012208E050EA010306D062
:1084F00030238DF804308DF8052002229146009B30
:1085000083F0080353EA0B030AD150EA010201D1B8
:10851000620705D530228DF804204FF001097F1E37
:108520003278582A04D039A20C920CAA02920BE09D
:108530003BA2F9E75B46009AF7F744FE0C9B9B5C75
:10854000029A521E0292137050EA0102F2D102986E
:1085500004A9081A00F1200B600702D524F4803426
:1085600000E001275F4502DDA7EB0B0000E00020E3
:1085700000EB0B01009003984944401A0390E0037C
:1085800006D453462146179A039800F0A9F90544EA
:10859000002706E001A85246C05D179990476D1C60
:1085A0007F1C4F45F6DBE0030CD553462146179A56
:1085B000039800F095F9054404E0302052461799DD
:1085C00090476D1C0099481E00900029F5DC08E0DA
:1085D0000298029952460078491C029117999047D7
:1085E0006D1CBBF10001ABF1010BF1DC5BE100F0B4
:1085F00065F90544761C307800287FF40DAE19B07B
:108600002846BDE8F08F00000928010030313233E0
:1086100034353637383961626364656600000000BE
:1086200030313233343536373839414243444546A8
:1086300000000000600700D4062708F1070020F0C2
:108640000700F0E80223804603F0004C5FEA0C00CC
:1086500001D097A009E0200501D596A005E0E0072C
:1086600001D095A001E0AFF24C001390307823F0D8
:10867000004365280CD006DC452809D046281DD0CB
:1086800047287FD13BE0662818D067287AD136E0AA
:108690000021112F01DB112000E0781CCDE9000141
:1086A00004A90CA8FFF7EEFCDDE90D010C9A4FF0D0
:1086B000000B07F10109109200914EE04FF00040CD
:1086C0000097CDE9011004A90CA8FFF7DBFCDDE958
:1086D0000D020C9B0F994FF0000B914610930092E6
:1086E00011B9791C00EB0109B7EB090003D4C0F103
:1086F000FF3B07F10109A9EB0700019042E0012FC0
:1087000000DA01270021112F01DD112000E0384699
:10871000CDE9000104A90CA8FFF7B4FCDDE90D01C7
:108720000C9A00914FF0000BB946109221070FD41C
:10873000009A4A4503DA914601E0A9F10109B9F12D
:10874000010F05DD109AA9F10101515C3029F4D027
:10875000B84202DA10F1040F03DA0121CDE9011069
:1087600010E0002803DC8344A9EB000102E0411C77
:10877000494500DD8946A0EB0B00401C01904FF0FD
:1087800000400290200705D40198484502DB4FF0D5
:10879000FF30019000208DF84B0002980DF14B073F
:1087A000B0F1004F25D002200C902B200D900298A4
:1087B00000280CDA404202902D200D9007E00A219B
:1087C0000298F8F735F83031029007F8011D0C993E
:1087D000481E0C900029F2DC02980028EFD1791E87
:1087E0000D980870307800F0200040F0450007F840
:1087F000020D11A8C01BC01D02901398007800B193
:10880000012000EB0901019801EBE071029801449D
:108810000398401A401E0390E00306D453462146B5
:10882000179A039800F05CF805441398007818B183
:108830005246179990476D1CE00323D553462146B5
:10884000179A039800F04CF805441BE0BBF1000FA9
:1088500007DB0098584504DD1098179910F80B00B5
:1088600001E0179930205246904701980BF1010B17
:10887000401E05F10105019004D12E2052461799A2
:1088800090476D1CB9F10001A9F10109DEDC05E09A
:1088900017F8010B5246179990476D1C0299481E14
:1088A00002900029F4DC53462146179A03989EE66D
:1088B0002D0000002B000000200000002DE9F041F9
:1088C000044600251E461746880404D405E03946B0
:1088D0002020B0476D1C641EF9D52846BDE8F08104
:1088E0002DE9F041044600251E469046C80301D5F7
:1088F000302700E02027880404D505E041463846AB
:10890000B0476D1C641EF9D52846BDE8F0810A68A1
:10891000531C0B601070704713B50C464FF47A73FC
:10892000012269460248FBF74BFF00981CBD00007E
:10893000E8040020FAF71AFCFEF776F9FDF7F6FADC
:10894000FDF7C8FAFDF7AAFCFDF7C4FCFDF73AFCF9
:10895000FDF7C8FBFDF75CFCFDF76EFAFDF77EFC4A
:10896000FDF7A2FBFDF7F6FBFDF72EFA00203549D7
:1089700008603549086035490860002210213448F4
:10898000FAF77AF8F8F7A6FB032232493248F9F7EA
:1089900039FCFCF73FFAFCF713FBF8F7D9FFFDF7BA
:1089A00001FDFDF74DFD2DA0FFF782F800203349B2
:1089B000087033490860FDF7ADFC32A0FFF778F886
:1089C0003C48FBF757F93C48FBF754F93B48FBF7A9
:1089D00051F93B48FBF74EF9FDF7D4F931E0FCF7CC
:1089E000BDFBF8F7AFFB3748007820B1FEF7D2FEA9
:1089F0000020344908703448007801280CD002283F
:108A000007D0032802D004280CD108E0F8F7D2FFE1
:108A10000CE0FDF76FF809E0F9F7D2F806E0FDF792
:108A2000F5FE03E003202849087000BF00BF274877
:108A3000008800F4004008B1F8F798FD0A20F9F723
:108A400005FFCCE724020020280200202C02002091
:108A5000001802401000002084020020496E697452
:108A600069616C697A696E67206F7A6F6E652063E1
:108A70006F6E74726F6C2E2E2E0A0000540100204F
:108A8000580100204F7A6F6E6520696E69746961C4
:108A90006C697A65642C2077616974696E672066F9
:108AA0006F722072656D6F746520636F6E74726F84
:108AB0006C0A0000100400205804002080030020ED
:108AC000C8030020540000202C0100209401002045
:108AD000000610160006101600000000000000003E
:108AE0000102030406070809000000000102030454
:108AF00004FA97999999D93FAF788E1DC571CC3FEB
:108B00009FC678D0099AC33F935555555555E53FB3
:108B1000599322942449D23FDE03CB966446C73F43
:108B200044523EDF12F1C23F00000000000000008E
:108B3000DDDDDDDDDCBBBBDDDDDDDDDDDDDDDDDDAA
:108B400098888888888888887777777777888888EA
:108B50008555555666666666666666666668888882
:108B60008333333222222222222222222228888D7B
:108B70007B225834223A25642C22583130223A255F
:108B8000642C22583132223A25642C225831332267
:108B90003A25642C22583134223A25642C2258314B
:108BA00035223A25642C22583138223A25642C2269
:108BB000583230223A25642C22583231223A256428
:108BC0002C225835223A252E32662C225832322257
:108BD0003A252E31662C22583233223A252E316620
:108BE0002C22583234223A25642C22583235223A2B
:108BF00025642C22583335223A25642C22583337E9
:108C0000223A25642C22583338223A25642C2258E3
:108C10003434223A25642C22583436223A25642CE6
:108C200022583437223A25642C22583439223A25E6
:108C3000642C22583530223A25642C2258353122B2
:108C40003A25642C22583532223A25642C22583594
:108C500033223A25642C22583534223A25642C22BA
:108C6000583535223A25642C22583536223A256467
:108C70002C22583537223A25642C22583538223A8E
:108C800025642C22583539223A25642C2258333059
:108C900030223A252E36662C2258303031223A22A4
:108CA0002573227D00000000C88C00080000002011
:108CB0003C020000780E0008208D00083C020020D5
:108CC000FC0F000068800008013032104201036D83
:108CD00024F42974329632283202320A9A1410E9A6
:108CE000203205DA19205A7834291C294029042910
:108CF0000C29241AA0094B400B281A680529080AD8
:108D00001CF0912923490B19010916B40910191BEC
:108D100070416E190409143001685A14F8013C00BE
:040000050800018965
:00000001FF
